:020000040800F2
:1000000000000824291300085D0F00085F0F000896
:10001000610F0008630F0008650F00080000000072
:10002000000000000000000000000000670F000852
:10003000690F0008000000006B0F00086D0F00083A
:100040007913000879130008791300087913000860
:100050007913000879130008791300087913000850
:10006000750F000879130008810F0008990F000828
:100070007913000879130008791300087913000830
:100080007913000879130008791300087913000820
:100090007913000879130008791300087913000810
:1000A0007913000879130008791300087913000800
:1000B000A90F0008791300087913000879130008C4
:1000C00079130008791300087913000879130008E0
:1000D00079130008B90F0008791300087913000894
:1000E0007913000879130008000000007913000854
:1000F00079130008791300087913000879130008B0
:10010000791300087913000879130008791300089F
:10011000791300087913000879130008791300088F
:10012000791300087913000879130008791300087F
:10013000791300087913000879130008791300086F
:1001400000000000000000000000000000000000AF
:10015000791300087913000879130008791300084F
:10016000791300087913000879130008791300083F
:10017000791300087913000879130008791300082F
:10018000791300087913000879130008791300081F
:10019000791300087913000879130008791300080F
:1001A00079130008791300087913000879130008FF
:1001B00079130008791300087913000879130008EF
:1001C00079130008791300087913000879130008DF
:1001D00079130008791300087913000879130008CF
:1001E00079130008791300087913000879130008BF
:1001F00079130008791300087913000879130008AF
:10020000791300087913000879130008791300089E
:10021000791300087913000879130008791300088E
:100220007913000879130008791300080000000012
:100230007913000879130008000000007913000802
:10024000791300087913000879130008791300085E
:10025000791300087913000879130008791300084E
:10026000791300087913000879130008791300083E
:1002700079130008791300087913000800000000C2
:1002800079130008791300087913000800000000B2
:080290000000000079130008D2
:1002980010B5054C237833B9044B13B10448AFF3B8
:1002A80000800123237010BD5408002400000000C2
:1002B8009C74000808B5034B1BB103490348AFF30E
:1002C800008008BD00000000580800249C74000845
:1002D80080F0004002E000BF81F0004142001FBFF3
:1002E8005FEA410392EA030F7FEA226C7FEA236CFC
:1002F8006AD04FEA1262D2EB1363C1BFD2184140F1
:1003080048404140B8BF5B42192B88BF704710F086
:10031800004F40F4000020F07F4018BF404211F029
:10032800004F41F4000121F07F4118BF494292EA91
:10033800030F3FD0A2F1010241FA03FC10EB0C00BD
:10034800C3F1200301FA03F100F0004302D549424A
:1003580060EB4000B0F5000F13D3B0F1807F06D3F7
:1003680040084FEA310102F10102FE2A51D2B1F1EF
:10037800004F40EBC25008BF20F0010040EA0300E4
:100388007047490040EB0000013A28BFB0F5000F64
:10039800EDD2B0FA80FCACF1080CB2EB0C0200FA1A
:1003A8000CF0AABF00EBC25052421843BCBFD04069
:1003B8001843704792F0000F81F4000106BF80F4E3
:1003C80000000132013BB5E74FEA41037FEA226CA6
:1003D80018BF7FEA236C21D092EA030F04D092F071
:1003E800000F08BF0846704790EA010F1CBF0020A5
:1003F800704712F07F4F04D1400028BF40F0004002
:10040800704712F100723CBF00F50000704700F021
:10041800004343F0FE4040F4000070477FEA226248
:1004280016BF08467FEA23630146420206BF5FEA19
:10043800412390EA010F40F4800070474FF0000319
:1004480004E000BF10F0004348BF40425FEA000CE0
:1004580008BF704743F0964301464FF000001CE088
:1004680050EA010208BF70474FF000030AE000BFDE
:1004780050EA010208BF704711F0004302D540421C
:1004880061EB41015FEA010C02BF8446014600208E
:1004980043F0B64308BFA3F18053A3F50003BCFAA9
:1004A8008CF2083AA3EBC25310DB01FA02FC634456
:1004B80000FA02FCC2F12002BCF1004F20FA02F25D
:1004C80043EB020008BF20F00100704702F1200250
:1004D80001FA02FCC2F1200250EA4C0021FA02F2B1
:1004E80043EB020008BF20EADC7070474FF0FF0CB6
:1004F8001CEAD0521EBF1CEAD15392EA0C0F93EAB1
:100508000C0F6FD01A4480EA010C400218BF5FEA52
:1005180041211ED04FF0006343EA501043EA5111C5
:10052800A0FB01310CF00040B1F5000F3EBF4900BF
:1005380041EAD3715B0040EA010062F17F02FD2AC3
:100548001DD8B3F1004F40EBC25008BF20F00100A6
:10055800704790F0000F0CF0004C08BF49024CEABD
:10056800502040EA51207F3AC2BFD2F1FF0340EA4F
:10057800C250704740F400004FF00003013A5DDCC0
:1005880012F1190FDCBF00F000407047C2F1000201
:10059800410021FA02F1C2F1200200FA02FC5FEAEE
:1005A800310040F1000053EA4C0308BF20EADC7038
:1005B800704792F0000F00F0004C02BF400010F4AA
:1005C800000F013AF9D040EA0C0093F0000F01F057
:1005D800004C02BF490011F4000F013BF9D041EA79
:1005E8000C018FE70CEAD15392EA0C0F18BF93EA7B
:1005F8000C0F0AD030F0004C18BF31F0004CD8D1A5
:1006080080EA010000F00040704790F0000F17BF2B
:1006180090F0004F084691F0000F91F0004F14D071
:1006280092EA0C0F01D142020FD193EA0C0F03D1C9
:100638004B0218BF084608D180EA010000F00040CC
:1006480040F0FE4040F40000704740F0FE4040F4A7
:10065800400070474FF0FF0C1CEAD0521EBF1CEA46
:10066800D15392EA0C0F93EA0C0F69D0A2EB030264
:1006780080EA010C49024FEA402037D04FF08053FE
:1006880043EA111143EA10130CF000408B4238BFC3
:100698005B0042F17D024FF4000C8B4224BF5B1AD1
:1006A80040EA0C00B3EB510F24BFA3EB510340EA1F
:1006B8005C00B3EB910F24BFA3EB910340EA9C00CD
:1006C800B3EBD10F24BFA3EBD10340EADC001B013D
:1006D80018BF5FEA1C1CE0D1FD2A3FF650AF8B42E1
:1006E80040EBC25008BF20F0010070470CF0004CEE
:1006F8004CEA50207F32C2BFD2F1FF0340EAC25019
:10070800704740F400004FF00003013A37E792F0D9
:10071800000F00F0004C02BF400010F4000F013A37
:10072800F9D040EA0C0093F0000F01F0004C02BF32
:10073800490011F4000F013BF9D041EA0C0195E79B
:100748000CEAD15392EA0C0F08D142027FF47DAF34
:1007580093EA0C0F7FF470AF084676E793EA0C0F24
:1007680004D14B023FF44CAF08466EE730F0004C22
:1007780018BF31F0004CCAD130F000427FF45CAFB2
:1007880031F000437FF43CAF5FE700BF42000ED278
:10079800B2F1FE4F0BD34FF09E03B3EB126209D4B4
:1007A8004FEA002343F0004323FA02F070474FF06A
:1007B8000000704712F1610F01D1420202D14FF0DF
:1007C800FF3070474FF00000704700BF53B94AB977
:1007D800002908BF00281CBF4FF0FF314FF0FF3041
:1007E80000F074B9ADF1080C6DE904CE00F006F81C
:1007F800DDF804E0DDE9022304B070472DE9F04795
:10080800089E0D4604468846002B4DD18A429446E0
:1008180068D9B2FA82F252B101FA02F3C2F12001A8
:1008280020FA01F10CFA02FC41EA030894404FEA6D
:100838001C45210CB8FBF5FE1FFA8CF705FB1E833F
:1008480041EA03430EFB07F199420BD91CEB030362
:100858000EF1FF3080F01E81994240F21B81AEF10B
:10086800020E63445B1AA4B2B3FBF5F005FB103328
:1008780044EA034400FB07F7A7420AD91CEB040427
:1008880000F1FF3380F00881A74240F205816444FB
:100898000238E41B40EA0E4000211EB1D440002378
:1008A800C6E90043BDE8F0878B4208D9002E00F066
:1008B800EE800021C6E900050846BDE8F087B3FAD6
:1008C80083F100294AD1AB4202D3824200F2F98077
:1008D800841A65EB030301209846002EE2D0C6E98E
:1008E8000048DFE702B9FFDEB2FA82F2002A40F0E0
:1008F8009180A1EB0C054FEA1C471FFA8CFE0121E1
:10090800B5FBF7F307FB1350250C45EA00450EFB32
:1009180003F0A84208D91CEB050503F1FF3802D201
:10092800A84200F2CB8043462D1AA4B2B5FBF7F0DB
:1009380007FB105544EA05440EFB00FEA64508D9FE
:100948001CEB040400F1FF3502D2A64500F2BB807F
:100958002846A4EB0E0440EA03409EE7C1F12007B5
:100968008B4022FA07FC4CEA030C20FA07F405FA3C
:1009780001F31C43FD404FEA1C4900FA01F3B5FBA3
:10098800F9F8200C1FFA8CFE09FB185540EA0545BA
:1009980008FB0EF0A84202FA01F20BD91CEB050580
:1009A80008F1FF3A80F08880A84240F28580A8F1DB
:1009B800020865442D1AA4B2B5FBF9F009FB1055DD
:1009C80044EA054500FB0EFEAE4508D91CEB0505BB
:1009D80000F1FF346CD2AE456AD90238654440EA6A
:1009E8000840A0FB0294A5EB0E05A542C846A64602
:1009F80056D353D05EB1B3EB080265EB0E0505FA8A
:100A080007F722FA01F3CD401F43C6E9007500211C
:100A1800BDE8F087C2F1200320FA03F10CFA02FCCA
:100A280025FA03F395400D434FEA1C471FFA8CFE45
:100A3800B3FBF7F107FB11302B0C43EA004301FB32
:100A48000EF0984204FA02F408D91CEB030301F1F2
:100A5800FF382FD298422DD9023963441B1AADB200
:100A6800B3FBF7F007FB103345EA034500FB0EF331
:100A7800AB4208D91CEB050500F1FF3816D2AB4292
:100A880014D902386544ED1A40EA014138E7314685
:100A9800304607E78646E5E61846FAE64B45A9D20A
:100AA800B9EB020864EB0C0E0138A3E74046EAE70D
:100AB800204694E74146D1E7D0467BE7023B6544B0
:100AC80032E7084609E76444023842E7704700BF46
:100AD80000B583B00B4BD3F8D82042F00102C3F81D
:100AE800D820D3F8D83003F001030193019B0022EA
:100AF80011460B2000F0BEFC0B2000F0F1FC03B007
:100B08005DF804FB0044025810B588B00024039433
:100B18000494059406940794194BD3F8E02042F006
:100B28008002C3F8E020D3F8E02002F080020192AE
:100B3800019AD3F8E02042F00102C3F8E020D3F88C
:100B4800E03003F001030293029B142303934FF454
:100B58008813049303A90B4802F0E6F822462146BD
:100B6800082000F087FC082000F0BAFC2246214645
:100B78000A2000F07FFC0A2000F0B2FC08B010BD8B
:100B88000044025800000258042800D07047084B5F
:100B98001B78002BFAD110B5064C236000F04CFCF2
:100BA8002060082000F0AAFC014B01221A7010BD39
:100BB800700800247808002410B584B0002400943C
:100BC80001940294039400F0BFFC01238DF80030D7
:100BD8008DF801404FF01052019212228DF8082032
:100BE8008DF809408DF80A4003228DF80B208DF806
:100BF8000C408DF80D308DF80E308DF80F4068469A
:100C080000F0C0FC042000F0ADFC04B010BD0000F2
:100C18000E4B1A680E4B1A70C2F307215970C2F3B3
:100C280007419970120EDA700A4A11681971116831
:100C3800090A59711168090C99711268120EDA7152
:100C48000D221A72FF225A72704700BF88080024CA
:100C58007C0800247408002472B6FEE700B59FB033
:100C68004C2200210BA805F08BFB2022002103A8B1
:100C780005F086FB022002F07BF900230093384B35
:100C8800DA6A22F00102DA62DB6A03F001030093F8
:100C9800344B9A6942F440429A619B6903F4404399
:100CA8000093009B2F4B9B6913F4005FFAD02E4BE7
:100CB800D3F8F42042F00202C3F8F420D3F8F43059
:100CC80003F002030193019B00230293254B9A69C9
:100CD80042F440429A619B6903F440430293204BDB
:100CE800DA6A42F00102DA62DB6A03F00103029376
:100CF800029B1C4B9B6913F4005FFAD001230B93F2
:100D08004FF480330C930223149315931693F02217
:100D18001792189319931A9308231B9300231C9373
:100D28001D930BA802F04EF9B0B93F230393032398
:100D380004930023059308230693402307930893FD
:100D48004FF4806209920A93042103A802F0A0FDDF
:100D580020B91FB05DF804FBFFF77EFFFFF77CFFAB
:100D680000040058004802580044025808B5FFF72C
:100D780023FF364B5B6913F4003F13D1BFF34F8F4A
:100D8800BFF36F8F314B0022C3F85022BFF34F8F50
:100D9800BFF36F8F5A6942F400325A61BFF34F8F25
:100DA800BFF36F8F294B5B6913F4803F27D1274B23
:100DB8000022C3F88420BFF34F8FD3F88040C4F3D8
:100DC8004E3000E01846C4F3C90243F6E07303EA64
:100DD800401343EA82731D49C1F860321346013A51
:100DE800002BF2D1431E0028ECD1BFF34F8F4B6983
:100DF80043F480334B61BFF34F8FBFF36F8F00F025
:100E0800E1FAFFF72BFFFFF77FFEFFF761FE00F027
:100E180059F900F0C9F90E4800F026F83C210D48B0
:100E280004F017F90B4B1B685A6A0B4B1A6000F059
:100E380003FB0A4B1B68C01A094B1860FFF7E8FE52
:100E48000A220849024804F001FAEBE700ED00E045
:100E580058090024940800248808002478080024ED
:100E6800740800247C08002408B5054B1860054B5D
:100E78001868002302221946806805F0D3FA08BDD5
:100E88008C0800241000002410B5013801280AD865
:100E980014464FF0FF3392B20748006805F028F86F
:100EA80040B9204610BD05F041FA092303604FF010
:100EB800FF30F7E70520F5E78C080024022801D861
:100EC8000020704708B505F031FA092303604FF098
:100ED800FF3008BD08B505F029FA092303604FF073
:100EE800FF3008BD08B548B94FF0FF330122084864
:100EF800006805F065F840B9012008BD05F016FA4C
:100F0800092303604FF0FF30F7E70520F5E700BF3E
:100F18008C08002408B5022804D84FF400534B600D
:100F2800002008BD05F002FA09230360F8E7000075
:100F380082B0074BD3F8F42042F00202C3F8F42041
:100F4800D3F8F43003F002030193019B02B0704719
:100F580000440258FEE7FEE7FEE7FEE7FEE77047BB
:100F68007047704708B500F05BFA08BD08B5042063
:100F780001F0EEFF08BD000008B5102001F0E8FF01
:100F8800024B1B6800225A6208BD00BF9408002467
:100F980008B5024801F02CFB08BD00BFE00800249A
:100FA80008B5024803F0A1FE08BD00BF940800245C
:100FB80008B5024804F00CFA08BD00BF580900241F
:100FC80010B503460C4A0D490D48006840B10C485D
:100FD80000680344521A934206D8094A136010BDA8
:100FE8000748084C0460F2E705F0A0F90C230360F9
:100FF8004FF0FF30F3E700BF0000082400040000B2
:1010080090080024400A0024244B1B6803F00F03B7
:10101800062B06D8214A136823F00F0343F0070371
:1010280013601F4B1A6842F001021A6000221A610D
:1010380019681C4A0A401A60184B1B6813F0080FFD
:1010480006D0164A136823F00F0343F00703136012
:10105800134B00229A61DA611A62134999621349A3
:10106800D962134919635A639963DA6319645A6434
:10107800196821F4802119601A660E4B1A680E4B04
:101088001340B3F1005F03D20C4B0122C3F80821CF
:101098000B4B43F2D2021A60704700BF0020005287
:1010A800004402587FEDF6EA000202020000FF0148
:1010B800800201010010005C0000FFFF0080005169
:1010C8000040005200B58DB02422002103A805F08D
:1010D80057F9002300930193029312484FF080427E
:1010E80002600322426083604FF0FF31C1600361F8
:1010F8008361039201230593099303A903F03CFF3D
:1011080050B90023009302936946064804F006F894
:1011180028B90DB05DF804FBFFF79EFDF1E7FFF776
:101128009BFDF6E79408002400B589B000230393DB
:1011380004930593069307930368B3F1804F02D095
:1011480009B05DF804FB164BD3F8E82042F0010221
:10115800C3F8E820D3F8E82002F001020192019ACE
:10116800D3F8E02042F00102C3F8E020D3F8E030E1
:1011780003F001030293029B0323039302230493C6
:101188000123079303A9074801F0CEFD0022114669
:101198001C2000F06FF91C2000F0A2F9D0E700BF76
:1011A800004402580000025808B51748174B03605E
:1011B8004FF4E133436000238360C36003610C2272
:1011C80042618361C36103624362836204F0E8FFA2
:1011D80070B900210C4805F05FF860B900210A4891
:1011E80005F07FF850B9084805F037F848B908BD48
:1011F800FFF732FDEDE7FFF72FFDEFE7FFF72CFDD7
:10120800F1E7FFF729FDF2E7580900240010014033
:1012180030B5B9B0044600213391349135913691F7
:101228003791C02202A805F0ABF822682F4B9A42EA
:1012380001D039B030BD01220023CDE9022302A834
:1012480002F0C2FD00284AD1294BD3F8F02042F021
:101258001002C3F8F020D3F8F02002F01002009238
:10126800009AD3F8E02042F00102C3F8E020D3F856
:10127800E03003F001030193019B4FF4C063339303
:10128800022334930025359536950723379333A9E0
:10129800184801F049FD1848184B03602A23436099
:1012A80040238360C5604FF48063036145618561B5
:1012B8004FF48073C3610562456200F0A3FB88B9EF
:1012C8000D4BE3679C6300221146252000F0D2F8FD
:1012D800252000F005F9E06F00F094FBA9E7FFF77F
:1012E800BBFCB1E7FFF7B8FCEAE700BF001001401C
:1012F8000044025800000258E00800241000024090
:101308000268054B9A4200D07047044B1A680132B4
:101318001A601B68F8E700BF00100140EC090024C0
:10132800DFF834D0FFF770FE0C480D490D4A002352
:1013380002E0D458C4500433C4188C42F9D30A4A82
:101348000A4C002301E013600432A242FBD304F0EC
:10135800F3FFFFF70BFD704700000824000000248E
:10136800540800240C750008540800243C0A002482
:10137800FEE70000104B1B780BB90120704710B531
:1013880004464FF47A70B0FBF3F30C4A1068B0FBD4
:10139800F3F000F0C5F868B90F2C01D901200AE074
:1013A800002221464FF0FF3000F064F8044B1C6027
:1013B800002000E0012010BD0800002400000024E7
:1013C8000C00002410B5032000F042F802F054F994
:1013D8000F498B69C3F303230E4AD35C03F01F0341
:1013E800D8408B6903F00F03D35C03F01F0320FA86
:1013F80003F3094A1360094B18600F20FFF7BAFF7F
:1014080010B10124204610BD0446FFF791FDF9E70D
:1014180000440258B47400080400002400000024AA
:10142800034B1B78034A11680B441360704700BFD5
:1014380008000024F0090024014B1868704700BF19
:10144800F0090024014B1868000C70470010005C7C
:101458000649CB6823F4E0631B041B0C000200F46C
:10146800E0600343024A1A43CA60704700ED00E097
:101478000000FA0500B5174BDB68C3F30223C3F17C
:10148800070CBCF1040F28BF4FF0040C03F1040E45
:10149800BEF1060F14D9033B4FF0FF3E0EFA0CFCC9
:1014A80021EA0C0199400EFA03F322EA03031943D7
:1014B800002807DB0901C9B2074B19545DF804FB82
:1014C8000023E9E700F00F000901C9B2034B1954E2
:1014D800F4E700BF00ED00E000E400E014ED00E0F8
:1014E800002807DB00F01F02400901239340024A4D
:1014F80042F82030704700BF00E100E000280CDB14
:1015080000F01F024009012393402030034A42F8AB
:101518002030BFF34F8FBFF36F8F704700E100E0BB
:101528000138B0F1807F0BD24FF0E0235861054AB3
:10153800F02182F823100020986107221A61704771
:101548000120704700ED00E0BFF35F8F044B5A6A3B
:1015580022F480325A620022C3F89420704700BFF8
:1015680000ED00E040F00100054BC3F894005A6A12
:1015780042F480325A62BFF34F8FBFF36F8F7047C8
:1015880000ED00E04378144AC2F89830D2F8A03051
:1015980023F00103C2F8A0304368C2F89C30017BF5
:1015A800C37A1B0643EA0173817A43EAC143417B4C
:1015B80043EA8143817B43EA4143C17B43EA0143D8
:1015C800417A43EA0123017A43EA410301780B4354
:1015D800C2F8A030704700BF00ED00E0F0B4876D9E
:1015E8000468664E664DAC4218BFB44242D0183506
:1015F800AC423FD01835AC423CD01835AC4239D05B
:101608001835AC4236D01835AC4233D01835AC4218
:1016180030D005F55675AC422CD01835AC4229D0DF
:101628001835AC4226D01835AC4223D01835AC4218
:1016380020D01835AC421DD01835AC421AD0183518
:10164800AC4217D04F4DAC4214D01435AC4211D037
:101658001435AC420ED01435AC420BD01435AC4224
:1016680008D01435AC4205D01435AC4202D014353C
:10167800AC4207D1446E856E6560C46E14B1046FC8
:10168800456F656004683D4E3D4DAC4218BFB4429D
:1016980052D01835AC424FD01835AC424CD0183522
:1016A800AC4249D01835AC4246D01835AC4243D08C
:1016B8001835AC4240D005F55675AC423CD01835CB
:1016C800AC4239D01835AC4236D01835AC4233D09C
:1016D8001835AC4230D01835AC422DD01835AC4254
:1016E8002AD01835AC4227D0264E274DAC4218BF19
:1016F800B44211D0254DAC420ED01435AC420BD0BB
:101708001435AC4208D01435AC4205D01435AC427F
:1017180002D01435AC4224D1C46D04F01F05012455
:10172800AC407C60046863608368402B20D0036809
:1017380099600368DA6014E0C46D04F01F0C3F245C
:1017480004FA0CF4BC6005682C6824F480242C602E
:10175800046863608368402B05D003689960036858
:10176800DA60F0BC704703689A600368D960F8E7EC
:1017780003689A600368D960F3E700BF100002406D
:1017880028000240085402581C5402583054025889
:1017980003682749274A934218BF8B422FD0183233
:1017A80093422CD01832934229D01832934226D033
:1017B8001832934223D01832934220D018329342E1
:1017C8001DD002F55672934219D01832934216D0A2
:1017D8001832934213D01832934210D018329342E1
:1017E8000DD0183293420AD01832934207D01832DB
:1017F800934204D023F0FF038365806D704710B4D3
:10180800D9B210390C4AA2FB0142C2F302120B4CA6
:10181800A25CC2655F2906D9094A1A40043282656A
:10182800806D10BC7047064A1A408265F8E700BF11
:101838001000024028000240ABAAAAAAC4740008FB
:1018480000FCFFFF83699BB9836A012B0AD0022B36
:1018580002D00BB100207047C36A13F0807F2AD1F1
:1018680000207047C36AB3F1C07F26D000207047BC
:10187800B3F5005F0AD0836A022B26D9032B26D141
:10188800C36A13F0807F24D100207047836A032B3A
:1018980003D8DFE803F01404140A00207047C36A71
:1018A80013F0807F0DD100207047C36AB3F1C07F69
:1018B80009D000207047012070470120704701209F
:1018C80070470120704701207047012070470020B1
:1018D800704701207047000003682249224A93425A
:1018E80018BF8B4228D01432934225D01432934229
:1018F80022D0143293421FD0143293421CD0143297
:10190800934219D01432934216D0DAB2103A1749DA
:10191800A1FB0212120916491944A8291FD9154B0F
:1019280013449B000366144B436602F01F02012315
:1019380003FA02F282667047DBB2083B0F4AA2FB49
:1019480003230F4A02EB1312920002660D4A426605
:10195800C3F30413012202FA03F3836670470832C3
:10196800DDE700BF085402581C540258ABAAAAAAC3
:10197800F0FBFDBF0082001080080240CDCCCCCC2B
:10198800009600168058025801794A1E072A2CD85A
:1019980030B40368154D164CA34218BFAB4218D09B
:1019A8001434A34215D01434A34212D01434A342E1
:1019B8000FD01434A3420CD01434A34209D01434E9
:1019C800A34206D00B4B0B449B00C3660A4B03672C
:1019D80005E00A4B0B449B00C366094B03670123D0
:1019E80003FA02F2426730BC704770470854025845
:1019F8001C5402583F820010400902403F960016CE
:101A08004059025870B50446FFF716FD002C00F047
:101A1800B681054623685349534A934218BF8B42FF
:101A28000CBF0122002250D030318B424DD01831EA
:101A38008B424AD018318B4247D018318B4244D060
:101A480018318B4241D018318B423ED001F5567186
:101A58008B423AD018318B4237D018318B4234D070
:101A680018318B4231D018318B422ED018318B422D
:101A78002BD018318B4228D018318B4225D03B49C6
:101A88003B4A934218BF8B4200F03181394A934256
:101A980000F02D811432934200F0298114329342D0
:101AA80000F025811432934200F0218114329342D0
:101AB80000F01D811432934200F0198140236365C0
:101AC800032384F8353001204AE0022184F83510D8
:101AD800002184F834107ABB274A93422CD018325C
:101AE800934229D01832934226D01832934223D0F9
:101AF8001832934220D0183293421DD002F5567204
:101B0800934219D01832934216D01832934213D008
:101B18001832934210D0183293420DD018329342A3
:101B28000AD01832934207D01832934204D01A6868
:101B380022F001021A6003E01A6822F001021A601A
:101B480023681A6812F0010F18D0FFF775FC431BC1
:101B5800052BF5D920236365032384F8353001204C
:101B680070BD00BF1000024028000240085402580F
:101B78001C54025830540258400002401A688148E8
:101B88001040A168E2680A4321690A4361690A436F
:101B9800A1690A43E1690A43216A0A430243616A67
:101BA800042900F099807849086878490140B1F122
:101BB800005F11D36168A1F12905A1F13F00032855
:101BC80088BF052D06D9A1F14700012802D94F3950
:101BD800032901D842F480121A602668756925F035
:101BE8000705636A1D43042B08D1A36A1D43E36AF2
:101BF80023B12046FFF726FE002872D175612046E2
:101C0800FFF7C6FDE36D03F01F023F239340836097
:101C180023685F495F4A934218BF8B4242D018320B
:101C280093423FD0183293423CD01832934239D075
:101C38001832934236D01832934233D01832934236
:101C480030D002F5567293422CD01832934229D0E4
:101C58001832934226D01832934223D01832934236
:101C680020D0183293421DD0183293421AD018321D
:101C7800934217D0484A934214D01432934211D059
:101C8800143293420ED0143293420BD01432934242
:101C980008D01432934205D01432934202D0143241
:101CA800934213D12046FFF717FEA368802B59D023
:101CB800236E22791A60636EA26E5A606368013BD4
:101CC800072B52D90023E36623676367002060650A
:101CD800012384F8353043E7E16A206B01430A4366
:101CE80061E740236365012084F8350038E7022264
:101CF80084F83520002284F834201A6827491140D6
:101D0800A268402A2CD0802A27D00022E06842EA24
:101D1800D002206942EAD002606942EAD002A06992
:101D280042EAD002E06942EAD002206A42EA10128E
:101D38000A431A6022681A4B13441A4AA2FB032367
:101D48001B099B00E3652046FFF722FDE26D02F0C8
:101D58001F0101228A4042605AE74FF48042D5E7CA
:101D68001022D3E700236360A2E72046FFF70CFEAA
:101D7800E36E00221A60236F626F5A60A6E70120A3
:101D8800EEE600BF3F8010FE0010005C0000FFFF81
:101D98001000024028000240085402580F00FEFFBD
:101DA800F8ABFDA7CDCCCCCC002800F03E8170B5B7
:101DB800044690F83400012800F03981012084F8A5
:101DC800340094F83500C0B2012807D04FF40063FE
:101DD8006365002384F83430012070BD022084F844
:101DE8003500002060652068924E934DA84218BFC8
:101DF800B0422FD01835A8422CD01835A84229D087
:101E08001835A84226D01835A84223D01835A8423C
:101E180020D01835A8421DD005F55675A84219D00E
:101E28001835A84216D01835A84213D01835A8423C
:101E380010D01835A8420DD01835A8420AD0183548
:101E4800A84207D01835A84204D0056825F0010536
:101E5800056003E0056825F0010505602046FFF7E9
:101E6800BDFB23687349744A934218BF8B4238D02C
:101E78001832934235D01832934232D018329342F6
:101E88002FD0183293422CD01832934229D01832CE
:101E9800934226D002F55672934222D018329342CA
:101EA8001FD0183293421CD01832934219D01832DE
:101EB800934216D01832934213D01832934210D05E
:101EC800183293420DD01A6822F00E0242F00A022C
:101ED8001A60236C93B12268136843F004031360FB
:101EE8000CE01A6822F01E0242F016021A60236CF7
:101EF80023B12268136843F00803136023684D492F
:101F08004D4A934218BF8B4242D0183293423FD079
:101F1800183293423CD01832934239D01832934247
:101F280036D01832934233D01832934230D002F56B
:101F3800567293422CD01832934229D018329342C9
:101F480026D01832934223D01832934220D0183228
:101F580093421DD0183293421AD01832934217D0A8
:101F6800364A934214D01432934211D01432934219
:101F78000ED0143293420BD01432934208D014324C
:101F8800934205D01432934202D0143293420ED1B8
:101F9800236E1A6812F4803F03D01A6842F48072E4
:101FA8001A60E36E1BB11A6842F480721A602368E3
:101FB8002049214A934218BF8B4230D018329342AD
:101FC8002DD0183293422AD01832934227D0183293
:101FD800934224D01832934221D0183293421ED013
:101FE80002F5567293421AD01832934217D018321B
:101FF800934214D01832934211D0183293420ED023
:10200800183293420BD01832934208D018329342B8
:1020180005D01A6842F001021A600020DDE61A684D
:1020280042F001021A600020D7E601207047022022
:10203800D3E600BF100002402800024008540258AE
:1020480070B50446FFF7F8F9002C00F091810546B9
:1020580094F83530DBB2022B06D080236365002369
:1020680084F83430012070BD23688C498C4A93422F
:1020780018BF8B4230D0183293422DD01832934279
:102088002AD01832934227D01832934224D01832DB
:10209800934221D0183293421ED002F556729342D1
:1020A8001AD01832934217D01832934214D01832EB
:1020B800934211D0183293420ED0183293420BD06B
:1020C8001832934208D01832934205D01A6822F089
:1020D8000E021A60266809E01A6822F01E021A60C9
:1020E8002268536923F080035361266823686B498B
:1020F8006B4A934218BF8B4242D0183293423FD06A
:10210800183293423CD01832934239D01832934255
:1021180036D01832934233D01832934230D002F579
:10212800567293422CD01832934229D018329342D7
:1021380026D01832934223D01832934220D0183236
:1021480093421DD0183293421AD01832934217D0B6
:10215800544A934214D01432934211D01432934209
:102168000ED0143293420BD01432934208D014325A
:10217800934205D01432934202D01432934204D1D0
:10218800226E136823F48073136023684349444A1A
:10219800934218BF8B422FD0183293422CD018325A
:1021A800934229D01832934226D01832934223D032
:1021B8001832934220D0183293421DD002F556723D
:1021C800934219D01832934216D01832934213D042
:1021D8001832934210D0183293420DD018329342DD
:1021E8000AD01832934207D01832934204D01A68A2
:1021F80022F001021A6003E01A6822F001021A6054
:10220800336813F0010F0ED0FFF716F9431B052BA7
:10221800F6D920236365032384F83530002384F836
:10222800343001201FE723681C491D4A934218BF18
:102238008B4239D01832934236D01832934233D079
:102248001832934230D0183293422DD0183293422C
:102258002AD01832934227D002F55672934223D0DF
:102268001832934220D0183293421DD0183293422C
:102278001AD01832934217D01832934214D0183219
:10228800934211D0183293420ED0A16DE36D03F042
:102298001F02012393404B600DE000BF1000024075
:1022A8002800024008540258A16DE36D03F01F0294
:1022B8003F2393408B6023682E492F4A934218BFCF
:1022C8008B4242D0183293423FD0183293423CD0CE
:1022D8001832934239D01832934236D0183293428A
:1022E80033D01832934230D002F5567293422CD034
:1022F8001832934229D01832934226D0183293428A
:1023080023D01832934220D0183293421DD018326D
:1023180093421AD01832934217D0184A934214D0D5
:102328001432934211D0143293420ED01432934295
:102338000BD01432934208D01432934205D0143291
:10234800934202D0143293420BD1636EA26E5A604C
:10235800E36E33B11A6822F480721A60236F626FD9
:102368005A60012384F83530002084F834007AE676
:10237800012078E610000240280002400854025864
:10238800002800F0298108B5024690F83530DBB204
:10239800022B03D080234365012008BD03689048C1
:1023A80090498B4218BF83420CBF0121002166D09F
:1023B8003030834263D01830834260D01830834273
:1023C8005DD0183083425AD01830834257D0183025
:1023D800834254D000F55670834250D0183083425F
:1023E8004DD0183083424AD01830834247D0183035
:1023F800834244D01830834241D0183083423ED0C3
:10240800183083423BD0196821F00E011960136817
:10241800A0F5956073498B4218BF83426AD0724910
:102428008B4267D018318B4264D018318B4261D00F
:1024380018318B425ED018318B425BD018318B42F9
:1024480058D001F556718B4254D018318B4251D077
:1024580018318B424ED018318B424BD018318B42F9
:1024680048D018318B4245D018318B4242D01831B0
:102478008B423FD0196821F0010119603EE0042029
:1024880082F8350081BB584A93422DD018329342C6
:102498002AD01832934227D01832934224D01832C7
:1024A800934221D0183293421ED002F556729342BD
:1024B8001AD01832934217D01832934214D01832D7
:1024C800934211D0183293420ED0183293420BD057
:1024D8001832934208D01832934205D01A6822F075
:1024E80001021A60002058E71A6822F001021A60F7
:1024F800002052E7196821F0010119601368384873
:1025080038498B4218BF834242D018318B423FD0A2
:1025180018318B423CD018318B4239D018318B425C
:1025280036D018318B4233D018318B4230D001F578
:1025380056718B422CD018318B4229D018318B42DE
:1025480026D018318B4223D018318B4220D0183135
:102558008B421DD018318B421AD018318B4217D0BC
:1025680022498B4214D014318B4211D014318B4242
:102578000ED014318B420BD014318B4208D0143159
:102588008B4205D014318B4202D014318B4217D1C3
:10259800116E0B6823F480730B60906DD36D03F09C
:1025A8001F0101238B404360536E916E5960D36EB7
:1025B80033B1196821F480711960136F516F596034
:1025C800012382F83530002382F83430136D2BB1A3
:1025D800104698470020E0E6012070470020DCE61E
:1025E80010000240280002404000024008540258EF
:1025F800F0B583B00446002301937D4B1D687D4BE5
:10260800A3FB0535AD0A876D3E68D7F800C003689F
:1026180079497A48834218BF8B420CBF01200020B9
:1026280061D0774A93425ED0183293425BD0183219
:10263800934258D01832934255D01832934252D010
:10264800183293424FD002F5567293424BD018324B
:10265800934248D01832934245D01832934242D020
:10266800183293423FD0183293423CD018329342EA
:1026780039D01832934236D06249634A934218BF20
:102688008B4212D0614A93420FD0143293420CD03D
:102698001432934209D01432934206D01432934232
:1026A80003D01432934240F061821A68E16D01F060
:1026B8001F010420884010EA0C0F00F0A78212F0D6
:1026C800040F00F0A382786012F4004F00F05A82E1
:1026D80012F4803F40F05082A36C002B00F0468239
:1026E8002046984742E2E26D02F01F0108228A4024
:1026F800324241D070BB424A93422BD018329342A7
:1027080028D01832934225D01832934222D018325A
:1027180093421FD0183293421CD002F5567293424E
:1027280018D01832934215D01832934212D018326A
:1027380093420FD0183293420CD01832934209D0EA
:102748001832934206D01832934203D01A68C2F363
:10275800C00202E01A68C2F380026AB11A6822F065
:1027680004021A60E36D03F01F0208239340BB6064
:10277800636D43F001036365E26D02F01F0226FA00
:1027880002F313F0010F47D023681B481B498B4203
:1027980018BF83423CD018318B4239D018318B4254
:1027A80036D018318B4233D018318B4230D01831A3
:1027B8008B422DD018318B422AD001F556718B42AD
:1027C80026D018318B4223D018318B4220D01831B3
:1027D8008B421DD018318B421AD018318B4217D03A
:1027E80018318B4214D018318B4211D01B6813E07A
:1027F80000000024B5814E1B100002402800024052
:1028080040000240085402581C54025830540258E0
:102818005B6913F0800F3BD1E36D03F01F030422C3
:1028280002FA03F3334240D02268964896498A4216
:1028380018BF824235D018318A4232D018318A42C4
:102848002FD018318A422CD018318A4229D0183119
:102858008A4226D018318A4223D001F556718A421D
:102868001FD018318A421CD018318A4219D0183129
:102878008A4216D018318A4213D018318A4210D0B1
:1028880018318A420DD018318A420AD013680CE0F8
:10289800012303FA02F2BA60636D43F00203636531
:1028A800BAE7126812F0020F3DD1E36D03F01F037F
:1028B800102202FA03F333425FD02268714872494A
:1028C8008A4218BF824234D018318A4231D0183136
:1028D8008A422ED018318A422BD018318A4228D009
:1028E80018318A4225D018318A4222D001F5567112
:1028F8008A421ED018318A421BD018318A4218D019
:1029080018318A4215D018318A4212D018318A42B9
:102918000FD018318A420CD018318A4209D0126877
:10292800C2F3800208E0BB60636D43F00403636593
:10293800BBE71268C2F3C002FAB1BB6023681A6829
:1029480012F4802F0DD01B6813F4002F04D1236CD0
:102958009BB12046984710E0A36C73B12046984776
:102968000BE01A6812F4807F03D11A6822F008027B
:102978001A60236C0BB120469847E36D03F01F03E0
:10298800202202FA03F3334200F0928022683D4885
:102998003D498A4218BF82422ED018318A422BD034
:1029A80018318A4228D018318A4225D018318A42F3
:1029B80022D018318A421FD018318A421CD001F522
:1029C80056718A4218D018318A4215D018318A4275
:1029D80012D018318A420FD018318A420CD01831DF
:1029E8008A4209D018318A4206D018318A4203D067
:1029F8001268C2F3400202E01268C2F30012002A11
:102A080056D0BB6094F83530DBB2042B0ED0236867
:102A18001A6812F4802F39D01B6813F4002F2CD1B8
:102A2800636C002B44D02046984741E02268136825
:102A380023F0160313602268536923F0800353615F
:102A4800236CB3B12268136823F008031360E36DA5
:102A580003F01F023F239340BB60012384F8353005
:102A6800002384F83430236D002B7FD0204698470C
:102A78007CE0A36C002BE5D1E9E7E36BC3B120460A
:102A8800984715E010000240280002401A6812F426
:102A9800807F09D11A6822F010021A60012384F895
:102AA8003530002384F83430E36B0BB12046984767
:102AB800636D002B5AD0636D13F0010F52D00423BD
:102AC80084F8353023689649964A934218BF8B425A
:102AD8002FD0183293422CD01832934229D0183272
:102AE800934226D01832934223D01832934220D0F2
:102AF800183293421DD002F55672934219D01832FB
:102B0800934216D01832934213D01832934210D001
:102B1800183293420DD0183293420AD01832934299
:102B280007D01832934204D01A6822F001021A60C2
:102B380003E01A6822F001021A60019B0133019335
:102B4800AB4204D823681B6813F0010FF5D1236842
:102B58001B6813F0010F0BD0032384F835300023D2
:102B680084F83430E36C0BB12046984703B0F0BDCD
:102B7800012384F83530F2E7236C002BF6D0204689
:102B88009847F3E712F0200F3AD123686449654A61
:102B9800934218BF8B422FD0183293422CD0183250
:102BA800934229D01832934226D01832934223D028
:102BB8001832934220D0183293421DD002F5567233
:102BC800934219D01832934216D01832934213D038
:102BD8001832934210D0183293420DD018329342D3
:102BE8000AD01832934207D01832934204D01A6898
:102BF80022F004021A6003E01A6822F008021A6040
:102C0800236C002BB2D020469847AFE702208840BB
:102C180010EA0C0F60D012F0020F5DD0786012F449
:102C2800004F0ED012F4803F05D1636C002B9DD06D
:102C3800204698479AE7E36B002B97D020469847A1
:102C480094E712F0200F40D123683549354A934262
:102C580018BF8B422FD0183293422CD0183293428F
:102C680029D01832934226D01832934223D01832F2
:102C7800934220D0183293421DD002F556729342E7
:102C880019D01832934216D01832934213D0183202
:102C9800934210D0183293420DD0183293420AD082
:102CA8001832934207D01832934204D01A6822F09F
:102CB8000A021A6003E01A6822F014021A6001235B
:102CC80084F83530002384F83430E36B002B3FF46C
:102CD8004DAF2046984749E7082000FA01F111EA6C
:102CE8000C0F3FF443AF12F0080F3FF43FAF1A68E0
:102CF80022F00E021A60E36D03F01F03012202FAAC
:102D080003F37B60626584F83520002384F834304F
:102D1800E36C002B3FF42AAF2046984726E700BF14
:102D2800100002402800024070B582B000236EE017
:102D380085685E000324B44025EA0405CC68B440E5
:102D48002C438460446824EA0C0C4C68C4F30014D7
:102D58009C4044EA0C0444606CE0DD08083550F8F7
:102D6800256003F007044FEA840C0F2404FA0CF4DE
:102D780026EA040E0C6904FA0CF444EA0E0440F83E
:102D880025406FE0092400E0002404FA0EF42C43E7
:102D98000CF1020C6B4D45F82C404FF0B0442568FF
:102DA800D44325EA0206D1F804C01CF4801F01D0E0
:102DB80042EA05064FF0B0452E606D6804EA050644
:102DC800D1F804C01CF4001F01D042EA05064FF0F8
:102DD800B0456E60D5F8845004EA0506D1F804C001
:102DE8001CF4003F01D042EA05064FF0B045C5F893
:102DF8008460D5F880502C404E6816F4803F01D08E
:102E080042EA05044FF0B042C2F8804001330A6834
:102E180032FA03F400F093804FF0010C0CFA03FC33
:102E28001CEA0202F2D04C6804F00304013C012CB5
:102E38007FF67EAF4C6804F00304032C0CD0C46802
:102E48005D004FF0030C0CFA05FC24EA0C0C8C68AE
:102E5800AC4044EA0C04C4604C6804F00304022C3F
:102E68003FF47BAF04684FEA430E4FF0030C0CFAB3
:102E78000EFC24EA0C0C4C6804F0030404FA0EF46B
:102E880044EA0C0404604C6814F4403FBED02E4C55
:102E9800D4F8F45045F00205C4F8F450D4F8F440DE
:102EA80004F002040194019C4FEA930C0CF1020512
:102EB800244C54F8255003F003044FEA840E0F24E1
:102EC80004FA0EF425EA0405204CA0423FF45CAF56
:102ED80004F58064A04222D004F58064A04220D08A
:102EE80004F58064A0421ED004F58064A0421CD082
:102EF80004F58064A0421AD004F58064A04218D07A
:102F080004F58064A04216D004F58064A04214D071
:102F180004F58064A0423FF435AF0A2435E7012464
:102F280033E7022431E703242FE704242DE705249F
:102F38002BE7062429E7072427E7082425E702B01A
:102F480070BD00BF00040058004402580000025839
:102F580008B54FF0B043D3F88830034200D108BD1C
:102F68004FF0B043C3F88800FDF70EFEF7E7000006
:102F7800134BDB6813F0040F07D1114BDB6803F028
:102F8800070383421AD00120704710B50C4AD36852
:102F980023F007031843D060FEF74EFA0446084BA7
:102FA8005B6813F4005F07D1FEF746FA001BB0F523
:102FB8007A7FF4D9012000E0002010BD002070477E
:102FC80000480258002800F0398338B504460368E1
:102FD80013F0010F25D0944A136903F03803926A5D
:102FE800102B15D0182B0FD06368B3F5803F3FD056
:102FF800002B53D18C4B1A6822F480321A601A685D
:1030080022F480221A6038E002F00302022AEBD18F
:10301800854B1B6813F4003F03D06368002B00F056
:103028000F83236813F0020F00F0A1807E4A136912
:10303800926A13F038035AD0182B55D0E368002B46
:1030480000F0DE8078490A6822F0190213430B6009
:10305800FEF7F2F90546744B1B6813F0040F40F0B5
:10306800AD80FEF7E9F9401B0228F4D90320EEE20F
:103078006D4A136843F48033136063682BB3FEF71B
:10308800DBF90546684B1B6813F4003FC9D1FEF70E
:10309800D3F9401B6428F5D90320D8E2B3F5A02F53
:1030A80009D0614B1A6822F480321A601A6822F437
:1030B80080221A60E1E75C4B1A6842F480221A60A9
:1030C8001A6842F480321A60D7E7FEF7B5F9054668
:1030D800554B1B6813F4003FA3D0FEF7ADF9401B16
:1030E8006428F5D90320B2E212F0030FA6D14E4BA3
:1030F8001B6813F0040F03D0E368002B00F0A282D2
:10310800494A136823F01903E1680B431360FEF77B
:1031180093F90546444B1B6813F0040F06D1FEF7DC
:103128008BF9401B0228F5D9032090E2FEF78AF9B3
:1031380041F20303984212D82269402A07D03A493B
:103148004B6823F47C3343EA02334B600FE0364A82
:10315800536823F47C3343F40033536007E0324A66
:10316800536823F0FE43216943EA016353602368EF
:1031780013F0100F00F088802B4A136903F038030E
:10318800926A082B56D0182B50D0E369002B00F018
:10319800B880254A136843F080031360FEF74CF9A2
:1031A8000546214B1B6813F4807F40F08880FEF7AA
:1031B80043F9401B0228F4D9032048E2FEF742F9FC
:1031C80041F20303984212D82269402A07D01649CF
:1031D8004B6823F47C3343EA02334B60C7E7124A57
:1031E800536823F47C3343F400335360BFE70E4A3B
:1031F800536823F0FE43216943EA01635360B6E74D
:10320800094A136823F001031360FEF715F9054610
:10321800054B1B6813F0040FA9D0FEF70DF9401BEE
:103228000228F5D9032012E20044025802F00302F2
:10323800012AAAD1A14B1B6813F4807F03D0E3694C
:10324800802B40F00182FEF7FDF841F2030398421B
:1032580012D8226A202A07D098494B6823F0F843ED
:1032680043EA82634B600FE0944A536823F0F843C3
:1032780043F08043536007E0904AD36823F07C53BF
:10328800216A43EA0163D360236813F0080F60D012
:103298006369002B49D0894A536F43F00103536790
:1032A800FEF7CAF80546854B5B6F13F0020F50D145
:1032B800FEF7C2F8401B0228F5D90320C7E1FEF744
:1032C800C1F841F20303984212D8226A202A07D093
:1032D8007A494B6823F0F84343EA82634B60D3E7AB
:1032E800764A536823F0F84343F080435360CBE7B2
:1032F800724AD36823F07C53216A43EA0163D3609E
:10330800C2E76E4A136823F080031360FEF794F84F
:1033180005466A4B1B6813F4807FB5D0FEF78CF81E
:10332800401B0228F5D9032091E1644A536F23F02A
:1033380001035367FEF780F80546604B5B6F13F097
:10334800020F06D0FEF778F8401B0228F5D90320B3
:103358007DE1236813F0200F29D0A3699BB1574A58
:10336800136843F480531360FEF766F80546534B21
:103378001B6813F4005F1AD1FEF75EF8401B0228A1
:10338800F5D9032063E14D4A136823F48053136091
:10339800FEF752F80546494B1B6813F4005F06D048
:1033A800FEF74AF8401B0228F5D903204FE12368AD
:1033B80013F0040F21D1636A002B00F047813F4AC4
:1033C800126902F03802182A00F0EE80022B79D038
:1033D8003A4A136823F080731360FEF72DF8044609
:1033E800364B1B6813F0007F00F0DC80FEF724F8F2
:1033F800001B0228F4D9032029E1314A136843F459
:1034080080731360FEF718F805462D4B1B6813F4FC
:10341800807F06D1FEF710F8401B6428F5D90320F9
:1034280015E1A368012B0AD00BBB244B1A6F22F0BD
:1034380001021A671A6F22F004021A6704E01F4A91
:10344800136F43F001031367A36833B3FDF7F4FF69
:1034580005461A4B1B6F13F0020FACD1FDF7ECFFBA
:10346800401B41F288339842F3D90320EFE0052B43
:1034780009D0124B1A6F22F001021A671A6F22F054
:1034880004021A67E0E70D4B1A6F42F004021A674C
:103498001A6F42F001021A67D6E7FDF7CDFF05461D
:1034A800064B1B6F13F0020F85D0FDF7C5FF401BBD
:1034B80041F288339842F3D90320C8E00044025807
:1034C80000480258694A136823F080731360FDF7B7
:1034D800B3FF0546654B1B6813F0007F06D0FDF768
:1034E800ABFF401B0228F5D90320B0E05F4B996A77
:1034F8005F4A0A40A16AE06A41EA00110A439A62F7
:10350800226B013AC2F30802616B0139490289B2A0
:103518000A43A16B0139090401F4FE010A43E16B76
:103528000139090601F0FE410A431A63DA6A22F0FA
:103538000102DA62596B4F4A0A40A16C42EAC102A1
:103548005A63DA6A22F00C02216C0A43DA62DA6AF8
:1035580022F00202616C0A43DA62DA6A42F48032CB
:10356800DA62DA6A42F40032DA62DA6A42F4802213
:10357800DA62DA6A42F00102DA621A6842F08072AC
:103588001A60FDF759FF0446384B1B6813F0007F9B
:1035980006D1FDF751FF001B0228F5D9032056E09C
:1035A800002054E0002052E0304A916A106B012B51
:1035B8004ED001F00303A26A93424BD1C1F3051127
:1035C800E36A994248D1C0F30802236B013B9A424F
:1035D80044D1C0F34622636B013B9A4240D1C0F309
:1035E8000642A36B013B9A423CD1C0F30660E36BF1
:1035F800013B984238D11D4B5B6BC3F3CC03A26CE3
:103608009A4201D1002022E0184AD36A23F001032C
:10361800D362FDF711FF0546FDF70EFFA842FBD068
:10362800124A516B134B0B40A16C43EAC10353631D
:10363800D36A43F00103D362002008E001207047F9
:10364800012004E0012002E0012000E0002038BD54
:103658000120FCE70120FAE70120F8E70120F6E75E
:103668000120F4E70120F2E70120F0E700440258C6
:103678000CFCFFFF0700FFFFF8B57E4B1B6903F04A
:103688003803102B00F0F280182B10D013B17A4CAD
:103698002046F8BD774B1B6813F0200F00F0E88038
:1036A800744B1868C0F3C100744CC440F0E7714B08
:1036B8009D6A05F003059C6AC4F30514D86A00F0F6
:1036C80001005B6BC3F3CC0303FB00F0FCF7B6FE11
:1036D8000646002CDCD0012D76D0022D00F0A48007
:1036E8000DB32046FCF7AAFE01466548FCF7B2FF79
:1036F8000446604B186BC0F30800FCF79FFE0546B4
:103708004FF064513046FCF7F1FE01462846FCF7BD
:10371800E5FD4FF07E51FCF7E1FD01462046FCF740
:10372800E5FE044671E0534B1B6813F0200F29D0C7
:10373800504F3B68C3F3C1035048D840FCF77EFEA6
:1037480005462046FCF77AFE01462846FCF782FF2C
:103758000446386BC0F30800FCF770FE05464FF0CE
:1037680064513046FCF7C2FE01462846FCF7B6FD18
:103778004FF07E51FCF7B2FD01462046FCF7B6FE3D
:10378800044642E02046FCF759FE01463D48FCF756
:1037980061FF0446374B186BC0F30800FCF74EFE78
:1037A80005464FF064513046FCF7A0FE0146284616
:1037B800FCF794FD4FF07E51FCF790FD0146204642
:1037C800FCF794FE044620E02046FCF737FE01464D
:1037D8002B48FCF73FFF0446264B186BC0F3080044
:1037E800FCF72CFE05464FF064513046FCF77EFE90
:1037F80001462846FCF772FD4FF07E51FCF76EFD3E
:1038080001462046FCF772FE04461A4B1B6BC3F3B5
:103818004623581CFCF712FE01462046FCF71AFF07
:10382800FCF7B4FF044633E72046FCF707FE0146E1
:103838001548FCF70FFF04460E4B186BC0F3080041
:10384800FCF7FCFD05464FF064513046FCF74EFE90
:1038580001462846FCF742FD4FF07E51FCF73EFD3D
:1038680001462046FCF742FE0446CEE7074C0FE728
:10387800024C0DE70044025800093D000090D003B7
:103888000024744A0024744C0024F44A00127A007C
:10389800002800F0328170B50D4604469B4B1B682A
:1038A80003F00F038B420BD2984A136823F00F03DF
:1038B8000B431360136803F00F038B4240F01F8122
:1038C800236813F0040F0CD02269914B9B6903F015
:1038D80070039A4205D98E498B6923F070031A4305
:1038E8008A61236813F0080F0CD06269884BDB6982
:1038F80003F070039A4205D98549CB6923F0700318
:103908001A43CA61236813F0100F0CD0A269804BC8
:10391800DB6903F4E0639A4205D97D49CB6923F456
:10392800E0631A43CA61236813F0200F0CD0E269E0
:10393800774B1B6A03F070039A4205D974490B6AE6
:1039480023F070031A430A62236813F0020F0CD0A5
:10395800E2686F4B9B6903F00F039A4205D96C49E3
:103968008B6923F00F031A438A61236813F0010F50
:1039780041D0674A936923F47063A1680B4393614C
:103988006368022B0AD0032B27D0012B2CD0604A66
:10399800126812F0040F06D10120ADE0126812F48B
:1039A800003F00F0AE805A490A6922F0070213432B
:1039B8000B61FDF741FD0646554B1B6903F03803C3
:1039C8006268B3EBC20F16D0FDF736FD801B41F2DB
:1039D80088339842F0D903208EE04D4A126812F0DD
:1039E800007FE0D1012087E0494A126812F4807F05
:1039F800D9D1012080E0236813F0020F0CD0E268CF
:103A0800434B9B6903F00F039A4205D240498B69E7
:103A180023F00F031A438A613C4B1B6803F00F0322
:103A2800AB420AD9394A136823F00F032B431360BA
:103A3800136803F00F03AB4265D1236813F0040F3A
:103A48000CD02269324B9B6903F070039A4205D26D
:103A58002F498B6923F070031A438A61236813F096
:103A6800080F0CD062692A4BDB6903F070039A4295
:103A780005D22749CB6923F070031A43CA6123682A
:103A880013F0100F0CD0A269214BDB6903F4E0633B
:103A98009A4205D21E49CB6923F4E0631A43CA61EE
:103AA800236813F0200F0CD0E269194B1B6A03F04E
:103AB80070039A4205D216490B6A23F070031A4321
:103AC8000A62FFF7D9FD12498B69C3F30323114A30
:103AD800D35C03F01F03D8408B6903F00F03D35C5A
:103AE80003F01F0320FA03F30B4A13600B4B186013
:103AF8000B4B1868FDF73EFC70BD01207047012094
:103B0800FAE70120F8E70120F6E700BF002000529D
:103B180000440258B4740008040000240000002483
:103B28000C00002408B5FFF7A7FD0B4A9369C3F3FF
:103B380003230A49CB5C03F01F0320FA03F39269BD
:103B480002F00F02885C00F01F0023FA00F0044A1C
:103B58001060044A136008BD00440258B474000899
:103B6800040000240000002408B5FFF7DBFF054B24
:103B7800DB69C3F30213044AD35C03F01F03D84084
:103B880008BD00BF00440258B474000808B5FFF728
:103B9800C9FF054BDB69C3F30223044AD35C03F076
:103BA8001F03D84008BD00BF00440258B474000881
:103BB800404B9B6A03F00303032B79D070B505468D
:103BC8000E463C4A136823F080631360FDF734FC0B
:103BD8000446384B1B6813F0006F06D0FDF72CFC29
:103BE800031B022BF5D9032070BD324B9A6A22F4CD
:103BF8007C32296842EA01329A626A68013AC2F361
:103C08000802A9680139490289B20A43E9680139F9
:103C1800090401F4FE010A4329690139090601F082
:103C2800FE410A439A63DA6A22F0C00269690A43CC
:103C3800DA62DA6A22F02002A9690A43DA62DA6AE9
:103C480022F01002DA62D96B1B4A0A40E96942EA9B
:103C5800C102DA63DA6A42F01002DA62C6B91A46B9
:103C6800DB6A43F40023D362124A136843F080638B
:103C78001360FDF7E1FB04460E4B1B6813F0006F61
:103C880014D1FDF7D9FB001B0228F5D90320ABE7B7
:103C9800012E05D0074AD36A43F40013D362E3E741
:103CA800044AD36A43F48013D362DDE700209BE71C
:103CB80001207047004402580700FFFF404B9B6AF1
:103CC80003F00303032B79D070B505460E463C4A32
:103CD800136823F080531360FDF7AEFB0446384B9E
:103CE8001B6813F0005F06D0FDF7A6FB031B022B31
:103CF800F5D9032070BD324B9A6A22F07C7229688C
:103D080042EA01529A626A68013AC2F30802A96853
:103D18000139490289B20A43E9680139090401F401
:103D2800FE010A4329690139090601F0FE410A43E7
:103D38001A64DA6A22F4406269690A43DA62DA6A62
:103D480022F40072A9690A43DA62DA6A22F48072FC
:103D5800DA62596C1B4A0A40E96942EAC1025A64AC
:103D6800DA6A42F48072DA62C6B91A46DB6A43F448
:103D78008003D362124A136843F080531360FDF73F
:103D88005BFB04460E4B1B6813F0005F14D1FDF774
:103D980053FB001B0228F5D90320ABE7012E05D001
:103DA800074AD36A43F08073D362E3E7044AD36ACD
:103DB80043F40003D362DDE700209BE7012070474E
:103DC800004402580700FFFFF8B50446036813F0E3
:103DD800006F30D0836EB3F5001F26D00ED8EBB13C
:103DE800B3F5801F07D102210830FFF7E1FE054631
:103DF80045B12E4621E0012635461EE0B3F5401FA9
:103E080009D10025984A136D23F44013A16E0B4382
:103E18001365002611E0012635460EE0924AD36A62
:103E280043F40033D3620025ECE702212830FFF782
:103E380045FF0546DCE700263546236813F4807FF6
:103E480014D0A36D042B32D8DFE803F003232A082B
:103E58000800854AD36A43F40033D36255BB824ACB
:103E6800136D23F00703A16D0B431365236813F447
:103E7800007F31D0E36D802B4CD020D8002B43D06D
:103E8800402B19D1002104F10800FFF791FE0546E7
:103E98001AE0002104F10800FFF78AFE0546DDE775
:103EA800002104F12800FFF709FF0546D6E701269F
:103EB8003546DBE72E46D9E7012635460CE0C02B10
:103EC80002D0B3F5807F1CD15DBB674A136D23F424
:103ED800E073E16D0B431365236813F4806F46D0DC
:103EE800D4F8A830B3F5800F39D01FD88BB3B3F509
:103EF800001F18D1002104F10800FFF759FE0546FC
:103F08001AE001263546E7E7574AD36A43F40033F7
:103F1800D362D9E7002104F12800FFF7CFFE054658
:103F2800D2E72E46D8E70126354620E0B3F5C00F84
:103F380002D0B3F5000F09D1C5B94B4A936D23F4EC
:103F48006003D4F8A8100B43936510E001263546AA
:103F58000DE0454AD36A43F40033D362ECE700210D
:103F680004F12800FFF7AAFE0546E5E72E46236878
:103F780013F4006F24D0D4F8AC30B3F1007F42D0F2
:103F88000ED8002B39D0B3F1807F06D1002104F17F
:103F98000800FFF70DFE054608E0012635460FE04C
:103FA800B3F1407F02D0B3F1806F23D1002D31D11E
:103FB8002D4A936D23F0E063D4F8AC100B4393655E
:103FC800236813F0007F2ED0E36C202B40D026D836
:103FD80033B1102B20D1244AD36A43F40033D3627F
:103FE800002D3CD1204AD36C23F03003E16C0B4305
:103FF800D36418E001263546E2E71B4AD36A43F446
:104008000033D362D2E7002104F12800FFF756FEFF
:104018000546CBE72E46D3E70126354603E0302B8D
:10402800DED001263546236813F4805F2DD0236E39
:10403800B3F5005F4FD019D8002B46D0B3F5805F99
:104048000FD1002104F10800FFF7B2FD054613E087
:10405800022104F10800FFF7ABFD0546C0E72E4634
:10406800E1E70126354610E000440258B3F5405F09
:1040780002D0B3F5804F25D1002D33D1774A136D87
:1040880023F4E043216E0B431365236813F4005FA8
:1040980038D0636EB3F5003F53D028D843B1B3F599
:1040A800803F21D1012104F10800FFF781FD054679
:1040B800002D4DD1694A136D23F4E023616E0B4343
:1040C80013651FE001263546DFE7644AD36A43F4E7
:1040D8000033D362D0E7002104F12800FFF7EEFD9A
:1040E8000546C9E72E46D0E7012635460AE0B3F56E
:1040F800802FDDD0B3F5A02FDAD0B3F5403FD7D06D
:1041080001263546236813F4804F31D0D4F8B030F7
:10411800B3F1005F45D020D843B1B3F1805F19D126
:10412800012104F10800FFF743FD0546002D3FD1AA
:104138004A4A936D23F0E043D4F8B0100B439365DB
:1041480016E0012104F12800FFF7B8FD0546AFE7A6
:104158002E46D7E7012635460AE0B3F1804FE5D071
:10416800B3F1A04FE2D0B3F1405FDFD0012635466E
:10417800236813F4004F09D0236FB3F1805F19D07F
:10418800B3F1005F24D0D3B101263546236813F07C
:10419800807F33D0A36C032B5BD8DFE803F02722A2
:1041A8005327012104F12800FFF788FD0546BDE7E4
:1041B8002E46DDE7294AD36A43F40033D36275B942
:1041C800264A136D23F04053216F0B431365DDE737
:1041D800012104F10800FFF7EBFC0546EFE72E4646
:1041E800D4E71E4AD36A43F40033D362A5BB1B4A03
:1041F800D36C23F00303A16C0B43D364236813F43B
:10420800800F2DD1236813F0010F00F0A580E36F14
:10421800282B00F29F80DFE803F08D9D9D9D9D9DDA
:104228009D9D879D9D9D9D9D9D9D969D9D9D9D9DD3
:104238009D9D8D9D9D9D9D9D9D9D8D9D9D9D9D9DC6
:104248009D9D8D00022104F10800FFF7B1FC054691
:10425800CCE701263546D1E72E46CFE70044025881
:10426800914A136843F480731360FDF7E5F8074635
:104278008D4B1B6813F4807F05D1FDF7DDF8C01B5B
:104288006428F5D90325002D4AD1884B1B6FD4F833
:10429800B420534013F4407F0CD0844B1A6F22F49F
:1042A8004072196F41F480311967196F21F4803118
:1042B80019671A67D4F8B430B3F5807F15D08DBB71
:1042C800D4F8B43003F44072B2F5407F1ED0774A78
:1042D800136923F47C53136174490B6FD4F8B42029
:1042E800C2F30B0213430B678CE7FDF7A5F80746EB
:1042F8006E4B1B6F13F0020FE1D1FDF79DF8C01B49
:1043080041F288339842F3D90325D8E76748026910
:1043180022F47C52664901EA131313430361DBE775
:104328002E466FE72E466DE7012104F10800FFF7DE
:104338003FFC0546E5B95D4A536D23F03803E16F4C
:104348000B43536508E0012104F12800FFF7B6FC90
:104358000546EFE701263546236813F0020F17D00C
:10436800A36F052B28D8DFE803F00B05200B0B0BF8
:104378002E46F1E7012104F10800FFF719FC054674
:10438800EDB94A4A536D23F00703A16F0B435365F8
:10439800236813F0040F23D0D4F89430052B45D8A4
:1043A800DFE803F0150F3D151515012104F128006C
:1043B800FFF784FC0546E3E701263546E8E72E4685
:1043C800E6E7012104F10800FFF7F2FB054685BB8B
:1043D800364A936D23F00703D4F894100B43936582
:1043E800236813F0200F34D0D4F89030B3F1005F75
:1043F8004ED023D843B1B3F1805F1CD1002104F122
:104408000800FFF7D5FB0546002D48D1274A536D14
:1044180023F0E043D4F890100B43536519E00121D1
:1044280004F12800FFF74AFC0546D0E70126354687
:10443800D6E72E46D4E7012635460AE0B3F1804F89
:10444800E2D0B3F1A04FDFD0B3F1405FDCD001265A
:104458003546236813F0400F37D0D4F89C30B3F5B5
:10446800006F53D026D843B1B3F5806F19D100211E
:1044780004F10800FFF79CFB0546002D4DD10B4ABF
:10448800936D23F4E053D4F89C100B4393651CE020
:10449800022104F12800FFF711FC0546B4E72E4677
:1044A800D7E70126354610E0004802580044025874
:1044B800CFFFFF00B3F5805FDFD0B3F5A05FDCD09E
:1044C800B3F5406FD9D001263546236813F0800F25
:1044D80033D0D4F8A030B3F5804F00F0A38021D8B2
:1044E80043B1B3F5005F1AD1002104F10800FFF7CA
:1044F8005FFB0546002D40F09C80814A936D23F4B4
:104508006043D4F8A0100B43936516E0022104F130
:104518002800FFF7D3FB0546AFE72E46D5E701266F
:1045280035460AE0B3F5004FE4D0B3F5204FE1D0AB
:10453800B3F5C04FDED001263546236813F0080FC7
:104548000CD0D4F88430B3F5805F74D06C4A536DC6
:1045580023F44053D4F884100B435365236813F0B5
:10456800100F0CD0D4F89830B3F5807F6CD0644A23
:10457800936D23F44073D4F898100B439365236824
:1045880013F4002F0BD0D4F8A430B3F5803F74D0C7
:10459800B3F5003F67D0002B5FD00126354623686E
:1045A80013F4802F0CD0D4F88830B3F5001F7CD0DA
:1045B800B3F5401F6FD0B3F5801F67D0012635468D
:1045C800236813F4803F08D0236D002B76D0B3F511
:1045D800803F00F0818001263546236813F0005F94
:1045E80040F08380236813F4003F00F08E80D4F8F5
:1045F8008030B3F5807F00F0EC8040F28380B3F523
:10460800007F03D0B3F5407F40F0E180002D40F0FB
:10461800E6803B4A536D23F44073D4F880100B4373
:10462800536572E0022104F12800FFF747FB0546B5
:1046380060E72E4681E7022104F12800FFF73EFBE0
:10464800002883D0012681E7022104F12800FFF722
:1046580035FB00288BD0012689E7002104F10800EA
:10466800FFF7A6FA05467DB9254A936D23F4403332
:10467800D4F8A4100B43936591E7022104F12800B4
:10468800FFF71CFB0546EEE72E4688E71C4AD36A6F
:1046980043F40033D3627DB9194A536D23F44013B0
:1046A800D4F888100B4353658AE7012104F12800E8
:1046B800FFF704FB0546EEE72E4681E7104AD36A6A
:1046C80043F40033D36275B90D4AD36C23F48033B5
:1046D800216D0B43D36480E7022104F10800FFF742
:1046E80067FA0546EFE72E4677E7022104F128002E
:1046F800FFF7E4FA00283FF475AF012672E700BF20
:1047080000440258002B81D00126236813F4801F2F
:1047180006D04F4A136D23F00043616F0B431365B6
:10472800236813F0805F07D0494A136923F4804354
:10473800D4F8B8100B431361236813F4001F06D094
:10474800434A136D23F08073E16E0B4313652368AE
:1047580013F0804F09D03E4B1A6922F400421A61C7
:104768001A69D4F8BC100A431A612368002B06DAC8
:10477800374AD36C23F04053616D0B43D3642368ED
:1047880013F4000F07D0324A536D23F44003D4F8D2
:104798008C100B435365636813F0010F21D16368D4
:1047A80013F0020F26D1636813F0040F2BD163684E
:1047B80013F0080F30D1636813F0100F35D1636818
:1047C80013F0200F3AD106B101263046F8BD012674
:1047D8009BE71F4AD36A43F40033D36216E72E4699
:1047E80093E7002104F10800FFF7E2F90028D6D08A
:1047F8000646D4E7012104F10800FFF7D9F900289B
:10480800D1D00646CFE7022104F10800FFF7D0F91E
:104818000028CCD00646CAE7002104F12800FFF79B
:104828004DFA0028C7D00646C5E7012104F1280043
:10483800FFF744FA0028C2D00646C0E7022104F177
:104848002800FFF73BFA0028BDD00646BBE700BFAB
:104858000044025808B5FFF765F9054B1B6AC3F316
:104868000213044AD35C03F01F03D84008BD00BFFD
:1048780000440258B47400082DE9F0410446864B00
:104888009D6A9E6AC6F30536D86AC0F30010DB6BD2
:10489800C3F3CC0303FB00F0FBF7D0FD002E00F0C0
:1048A800F58005F003050746012D79D0022D00F0AB
:1048B800CB800DB33046FBF7C1FD01467748FBF7C7
:1048C800C9FE0546744B986BC0F30800FBF7B6FDAC
:1048D80006464FF064513846FBF708FE014630465D
:1048E800FBF7FCFC4FF07E51FBF7F8FC014628462D
:1048F800FBF7FCFD054674E0674B1B6813F0200FBF
:104908002CD0DFF89481D8F80030C3F3C103644891
:10491800D840FBF793FD05463046FBF78FFD01466F
:104928002846FBF797FE0546D8F83800C0F308007C
:10493800FBF784FD06464FF064513846FBF7D6FD79
:1049480001463046FBF7CAFC4FF07E51FBF7C6FC28
:1049580001462846FBF7CAFD054642E03046FBF70C
:104968006DFD01464F48FBF775FE05464A4B986BAF
:10497800C0F30800FBF762FD06464FF06451384665
:10498800FBF7B4FD01463046FBF7A8FC4FF07E511B
:10499800FBF7A4FC01462846FBF7A8FD054620E0E6
:1049A8003046FBF74BFD01463C48FBF753FE0546F6
:1049B800394B986BC0F30800FBF740FD06464FF0F3
:1049C80064513846FBF792FD01463046FBF786FCFA
:1049D8004FF07E51FBF782FC01462846FBF786FD27
:1049E80005462D4EB06BC0F34620FBF727FD4FF070
:1049F8007E51FBF773FC01462846FBF72BFEFBF7BD
:104A0800C5FE2060B06BC0F30640FBF717FD4FF002
:104A18007E51FBF763FC01462846FBF71BFEFBF7BC
:104A2800B5FE6060B06BC0F30660FBF707FD4FF0A2
:104A38007E51FBF753FC01462846FBF70BFEFBF7BC
:104A4800A5FEA060BDE8F0813046FBF7F7FC014603
:104A58001548FBF7FFFD05460F4B986BC0F30800A0
:104A6800FBF7ECFC06464FF064513846FBF73EFD79
:104A780001463046FBF732FC4FF07E51FBF72EFC27
:104A880001462846FBF732FD0546AAE700232360C6
:104A98006360A360D6E700BF004402580024744A4C
:104AA8000090D0030024744C0024F44A2DE9F0410E
:104AB8000446864B9D6A9E6AC6F30556D86AC0F3BB
:104AC80000205B6CC3F3CC0303FB00F0FBF7B6FCE0
:104AD800002E00F0F58005F003050746012D79D07A
:104AE800022D00F0CB800DB33046FBF7A7FC014642
:104AF8007748FBF7AFFD0546744B186CC0F3080008
:104B0800FBF79CFC06464FF064513846FBF7EEFC79
:104B180001463046FBF7E2FB4FF07E51FBF7DEFB28
:104B280001462846FBF7E2FC054674E0674B1B6824
:104B380013F0200F2CD0DFF89481D8F80030C3F39D
:104B4800C1036448D840FBF779FC05463046FBF7BB
:104B580075FC01462846FBF77DFD0546D8F8400060
:104B6800C0F30800FBF76AFC06464FF0645138466C
:104B7800FBF7BCFC01463046FBF7B0FB4FF07E511B
:104B8800FBF7ACFB01462846FBF7B0FC054642E0C4
:104B98003046FBF753FC01464F48FBF75BFD0546E3
:104BA8004A4B186CC0F30800FBF748FC06464FF068
:104BB80064513846FBF79AFC01463046FBF78EFBFA
:104BC8004FF07E51FBF78AFB01462846FBF78EFC27
:104BD800054620E03046FBF731FC01463C48FBF730
:104BE80039FD0546394B186CC0F30800FBF726FC65
:104BF80006464FF064513846FBF778FC01463046CC
:104C0800FBF76CFB4FF07E51FBF768FB014628462B
:104C1800FBF76CFC05462D4E306CC0F34620FBF7C5
:104C28000DFC4FF07E51FBF759FB01462846FBF778
:104C380011FDFBF7ABFD2060306CC0F30640FBF7BD
:104C4800FDFB4FF07E51FBF749FB01462846FBF779
:104C580001FDFBF79BFD6060306CC0F30660FBF75D
:104C6800EDFB4FF07E51FBF739FB01462846FBF779
:104C7800F1FCFBF78BFDA060BDE8F0813046FBF747
:104C8800DDFB01461548FBF7E5FC05460F4B186CA4
:104C9800C0F30800FBF7D2FB06464FF064513846D4
:104CA800FBF724FC01463046FBF718FB4FF07E511A
:104CB800FBF714FB01462846FBF718FC0546AAE754
:104CC800002323606360A360D6E700BF0044025856
:104CD8000024744A0090D0030024744C0024F44A41
:104CE8007047704770477047704770B5044603684F
:104CF800DE681D6915F0020F10D016F0020F0DD0F6
:104D08006FF002021A610123037703689B6913F0AD
:104D1800030F64D0FFF7E6FF0023237715F0040F95
:104D280012D016F0040F0FD023686FF004021A6136
:104D38000223237723689B6913F4407F55D02046CC
:104D4800FFF7D0FF0023237715F0080F12D016F0D5
:104D5800080F0FD023686FF008021A610423237725
:104D68002368DB6913F0030F46D02046FFF7BAFF2C
:104D78000023237715F0100F12D016F0100F0FD064
:104D880023686FF010021A61082323772368DB6910
:104D980013F4407F37D02046FFF7A4FF0023237782
:104DA80015F0010F02D016F0010F33D115F4025F90
:104DB80002D016F0800F35D115F4807F02D016F09E
:104DC800800F37D115F0400F02D016F0400F39D1BF
:104DD80015F0200F02D016F0200F3BD170BDFFF761
:104DE80080FF2046FFF77FFF96E72046FFF779FF11
:104DF8002046FFF778FFA5E72046FFF772FF204619
:104E0800FFF771FFB4E72046FFF76BFF2046FFF777
:104E18006AFFC3E723686FF001021A612046FFF7B3
:104E28005FFFC3E723686FF402521A61204600F05F
:104E3800C6F9C1E723686FF480721A61204600F052
:104E4800BFF9BFE723686FF040021A612046FFF7F9
:104E58004BFFBDE723686FF020021A61204600F07F
:104E6800ADF9BBE730B503683D4A904214BF4FF037
:104E7800000E4FF0010EB0F1804F14BF72464EF095
:104E88000102AAB9374CA04214BF00240124364DB0
:104E9800A8420DD064B904F1804404F58234A042DC
:104EA80014BF0024012405F50065A84200D01CB1F8
:104EB80023F070034C68234312BB2A4A904214BF64
:104EC80000220122284CA0421AD0CAB902F180421D
:104ED80002F58232904214BF0022012204F50064D8
:104EE800A0420DD062B9214A904214BF002201228B
:104EF80004F59A34A04203D012B91D4A904204D155
:104F080023F4407CCB6843EA0C0323F080034A690E
:104F1800134303608A68C2620A688262154A904233
:104F280014BF73464EF0010363B9104B984214BF87
:104F38000023012302F57052904203D013B90C4BA1
:104F4800984201D10B69036301234361036913F09C
:104F5800010F03D0036923F00103036130BD00BFD3
:104F680000000140000800400004004000440140E7
:104F78000048014000040140002852D070B50D4699
:104F8800044690F83D30002B46D0022384F83D308B
:104F980022689168244B0B409360214651F8040B1A
:104FA800FFF760FF206881688369026A2E680E43F4
:104FB8001E491940AB68D5F818C043EA0C2343EAE8
:104FC800010C1B4B0CEA0303E968D5F81CC041EA45
:104FD8000C2119432B6A1B03D5F810C043EA0C13A4
:104FE8000B4322F0AA016A686D6942EA05120A4376
:104FF800866021688B6123681A62012384F848302F
:1050080084F83E3084F83F3084F8443084F84530E2
:1050180084F83D30002070BD80F83C30FCF784F8FF
:10502800B3E70120704700BFF8BFFEFFFCFCFFFF9D
:105038000303FFFF01F01F01012303FA01FC036AC8
:1050480023EA0C030362036A02FA01F10B430362C9
:10505800704738B5044690F83E30DBB290F83F20F0
:105068005FFA82FC90F84420D0B294F845200D46AF
:10507800B1B9012808BF012B47D1022384F83E307B
:1050880084F844307DB3042D39D0012200212068F2
:10509800FFF7D0FF012204212068FFF7CBFF27E0AC
:1050A800D2B2042914D0BCF1010F08BF012B30D1B2
:1050B800013A18BF012201282DD162BB022384F8CE
:1050C8003E3084F83F3084F8443084F84530D9E7DE
:1050D800012A08BFBCF1010F19D1022384F83F301F
:1050E80084F84530CEE7012200212068FFF7A2FFAF
:1050F8002268136843F001031360002038BD0122C1
:1051080004212068FFF796FFF2E70120F6E7012067
:10511800F4E70120F2E70120F0E7000090F83C30C6
:10512800012B45D070B4012380F83C30022380F86D
:105138003D3003685A689C681E4E1F4DAB4218BF2D
:10514800B34203D122F470024D682A4322F0700260
:105158000D682A435A600368164AB3F1804F18BF96
:10516800934217D0A2F57C42934213D002F5806295
:1051780093420FD002F5806293420BD002F5784239
:10518800934207D0A2F56C42934203D002F59432C1
:10519800934204D124F080048A6814439C6001235C
:1051A80080F83D30002380F83C30184670BC7047CA
:1051B800022070470000014000040140704770471A
:1051C8007047026852E8003F23F0C00342E800310C
:1051D8000029F6D1026802F1080353E8003F23F4DE
:1051E8000003083242E800310029F3D12023C0F837
:1051F80088307047026852E8003F23F4907342E811
:1052080000310029F6D1026802F1080353E8001FB3
:105218000D4B0B40083242E800310029F3D1C36E30
:10522800012B06D02023C0F88C300023C3664367C7
:105238007047026852E8003F23F0100342E800314B
:105248000029F6D1EEE700BFFEFFFFEF1346D0F8C6
:105258008820202A3DD110B50446002B18BF00290C
:1052680039D00165A0F85430A0F856300022C0F8B3
:1052780090202122C0F88820C26FCAB11749D16393
:10528800C26F17491164C26F1649D164C26F0021F9
:10529800116502682832016DC06FFCF785FD38B1D1
:1052A8001023C4F890302023C4F8883001200FE080
:1052B800236840221A62226802F1080353E8003F7B
:1052C80043F08003083242E800310029F3D100207E
:1052D80010BD022070470120FAE700BFF152000814
:1052E8005D5300086953000808B50346806BDB6905
:1052F800B3F5807F18D00023A0F85630026802F179
:10530800080353E8003F23F08003083242E80031E5
:105318000029F3D1026852E8003F43F0400342E815
:1053280000310029F6D108BDFBF7EAFFFBE708B515
:10533800026852E8003F23F0400342E800310029A8
:10534800F6D12023C0F8883000238367FBF7D8FF05
:1053580008BD704708B5806BFFF7FBFF08BD7047B5
:1053680038B5846BD4F88820D4F88C5023689B68AF
:1053780013F0800F01D0212A10D023689B6813F006
:10538800400F01D0222D10D0D4F8903043F01003F4
:10539800C4F890302046FFF7E2FF38BD0023A4F898
:1053A80056302046FFF70DFFE7E70023A4F85E30EC
:1053B8002046FFF71FFFE7E708B5806B0023A0F83A
:1053C8005E30A0F85630FFF7CAFF08BD70470000EE
:1053D80070B504460168CB6908688D6840F60F020D
:1053E8001A4008D113F0200F05D010F0200F34D147
:1053F80015F0805F31D12AB18B4A2A4033D18B4EC8
:10540800304230D1E26E012A00F0C68013F4801FCA
:1054180003D015F4800F40F09B8113F0800F07D064
:1054280010F0800F40F09B8115F4000F40F0978139
:1054380013F0400F03D010F0400F40F0978113F4A1
:10544800000F03D010F0804F40F0948113F0807F5C
:1054580002D00028C0F2928170BD636F002BFBD090
:1054680020469847F8E713F0010F09D010F4807F21
:1054780006D001260E62D4F890103143C4F890107B
:1054880013F0020F0BD015F0010F08D02168022687
:105498000E62D4F8901041F00401C4F8901013F093
:1054A800040F0BD015F0010F08D0216804260E62F6
:1054B800D4F8901041F00201C4F8901013F0080FCE
:1054C8000BD010F0200F00D13AB1226808211162E8
:1054D800D4F890200A43C4F8902013F4006F0CD03D
:1054E80010F0806F09D022684FF400611162D4F87F
:1054F800902042F02002C4F89020D4F89020002A8E
:10550800AAD013F0200F09D010F0200F02D115F007
:10551800805F03D0636F0BB120469847D4F8902082
:1055280023689B6813F0400F02D112F0280F2CD08B
:105538002046FFF75FFE23689B6813F0400F20D0DA
:10554800226802F1080353E8003F23F040030832C1
:1055580042E800310029F3D1D4F880306BB1344AE5
:105568001A65D4F88000FCF70BFF00283FF474AFED
:10557800D4F88000036D98476EE72046FFF7EFFEEA
:105588006AE72046FFF7EBFE66E72046FFF7E7FEEF
:105598000023C4F890305FE713F0100F3FF436AFE4
:1055A80010F0100F3FF432AF10230B6223689B6892
:1055B80013F0400F00F09280D4F8802013681D4843
:1055C8001D498B4218BF834238D018318B4235D0E1
:1055D80018318B4232D018318B422FD018318B4280
:1055E8002CD018318B4229D018318B4226D001F5A6
:1055F80056718B4222D018318B421FD018318B4202
:105608001CD018318B4219D018318B4216D0183162
:105618008B4213D018318B4210D018318B420DD0E9
:105628005B689BB20CE000BF010000102001000481
:10563800C153000810000240280002405B689BB27A
:10564800002B3FF409AFB4F85C1099427FF604AF21
:10565800A4F85E30D369B3F5807F32D0226852E86F
:10566800003F23F4807342E800310029F6D1226814
:1056780002F1080353E8003F23F00103083242E82F
:1056880000310029F3D1226802F1080353E8003FF2
:1056980023F04003083242E800310029F3D12023E7
:1056A800C4F88C300023E366226852E8003F23F0F8
:1056B800100342E800310029F6D1D4F88000FCF745
:1056C800BFFC02232367B4F85C10B4F85E309BB2C9
:1056D800C91A89B22046FFF779FEBDE6B4F85C1016
:1056E800B4F85E309BB2C91A89B2B4F85E309BB286
:1056F800002B3FF4B1AE00293FF4AEAE226852E869
:10570800003F23F4907342E800300028F6D1226865
:1057180002F1080353E8000F1A4B0340083242E82D
:1057280000300028F3D12023C4F88C300023E3662E
:105738006367226852E8003F23F0100342E8003014
:105748000028F6D1022323672046FFF73FFE83E6B1
:105758004FF480130B62204600F07CFD7CE6A36FBB
:10576800002B3FF479AE2046984775E62046FFF7B0
:10577800DEFD71E6204600F06FFD6DE6204600F084
:105788006AFD69E6FEFFFFEF70B586B00446016862
:1057980083680269134342691343C2691343086863
:1057A800884A024013430B602268536823F440532D
:1057B800E1680B435360A1692268834B9A4201D088
:1057C800236A19439068814B03400B439360226816
:1057D800D36A23F00F03616A0B43D36222687C4BC0
:1057E8009A4221D07B4B9A4200F08C807A4B9A42A5
:1057F80000F0A280794B9A4200F0B580784B9A422B
:1058080000F0C880774B9A4200F0F480764B9A42B9
:1058180000F01981754B9A4200F02C816A4B9A422C
:1058280000F03F81802333E0714B5B6D03F0380358
:10583800282B65D8DFE813F02900640064006400B1
:1058480064006400640064004D0164006400640046
:1058580064006400640064002B0064006400640059
:1058680064006400640064005E0064006400640016
:105878006400640064006400600064006400640004
:1058880064006400640064006200012300E00823EF
:105898004D498A4200F02F81E069B0F5004F00F0D1
:1058A800AF81202B00F20782202B00F25182DFE823
:1058B80013F01E0224024F024F0227024F024F022A
:1058C8004F022C024F024F024F024F024F024F026B
:1058D8004F0231024F024F024F024F024F024F0256
:1058E8004F024F024F024F024F024F024F024F0228
:1058F8004F023D021023CBE72023C9E74023C7E727
:105908008023C5E73A4B5B6D03F00703052B11D8DD
:10591800DFE813F00600E10008000A000C000E00A2
:105928000023B5E70823B3E71023B1E72023AFE747
:105938004023ADE78023ABE72D4B5B6D03F00703F6
:10594800052B0ED8DFE803F003C90507090B002370
:105958009EE708239CE710239AE7202398E7402333
:1059680096E7802394E7224B5B6D03F00703052B32
:105978000ED8DFE803F003B40507090B002387E717
:10598800082385E7102383E7202381E740237FE767
:1059980080237DE7164B5B6D03F00703052B0ED8BC
:1059A800DFE803F0039F0507090B002370E70823CE
:1059B8006EE710236CE720236AE7402368E780231B
:1059C80066E700BFF369FFCF000C0058FFF4FF1132
:1059D800001001400044004000480040004C0040D6
:1059E800005000400014014000780040007C004056
:1059F800004402587D4B5B6D03F03803282B20D8F8
:105A0800DFE803F0151F1F1F1F1F1F1F711F1F1F18
:105A18001F1F1F1F171F1F1F1F1F1F1F191F1F1F9C
:105A28001F1F1F1F1B1F1F1F1F1F1F1F1D000123BD
:105A38002EE708232CE710232AE7202328E7402312
:105A480026E7802324E7694B5B6D03F00703052BEA
:105A58000ED8DFE803F0034A0507090B002317E710
:105A6800082315E7102313E7202311E740230FE746
:105A780080230DE75D4B5B6D03F00703052B0ED804
:105A8800DFE803F003350507090B002300E70823C7
:105A9800FEE61023FCE62023FAE64023F8E68023FE
:105AA800F6E603F50E339B6D03F00703052B0ED8BE
:105AB800DFE803F0031F0507090B0223E8E60823C4
:105AC800E6E61023E4E62023E2E64023E0E680232E
:105AD800DEE60423DCE60423DAE60423D8E604231E
:105AE800D6E60423D4E60423D2E60423D0E604232E
:105AF800CEE60423CCE6202B27D8022BC0F01A814F
:105B0800023B1E2B00F21881DFE813F0500016014B
:105B180056001601160116015B0016011601160142
:105B2800160116011601160160001601160116016C
:105B380016011601160116011601160116011601A5
:105B480016011601160116016C00402B2CD14FF4DA
:105B58000040626A264B33F81220B0FBF2F3656806
:105B680005EB4501994200F2E980B3EB053F00F2ED
:105B7800E780002633463146FAF728FE090241EA53
:105B8800106100026B08C0182A46334641F1000133
:105B9800FAF71CFEA0F54072164B9A4200F2D2802A
:105BA8002368D8603046D4E00120D2E0FEF752FEE8
:105BB8000028CED10020CCE003A8FEF75DFE0498B3
:105BC800F6E76846FEF772FF0198F1E7074B1B6896
:105BD80013F0200F08D0054B1B68C3F3C103064818
:105BE800D840E5E70548B4E70348B2E7004402585F
:105BF800CC740008FFFC0F000090D00300093D00A2
:105C0800202B15D8202B00F29F80DFE803F03137D6
:105C18009D9D3A9D9D9D3F9D9D9D9D9D9D9D449DC6
:105C28009D9D9D9D9D9D9D9D9D9D9D9D9D9D500086
:105C3800402B1BD1626A4D4B33F81230B0FBF3F0A6
:105C48006268530803EB4000B0FBF2F0A0F11002C9
:105C58004FF6EF739A4279D883B223F00F03C0F35B
:105C6800420018432368D860002072E0012070E0E9
:105C7800FDF77AFF0028DDD100206AE0FDF786FFF6
:105C8800F8E703A8FEF7F8FD0498F3E76846FEF77F
:105C98000DFF0198EEE7364B1B6813F0200F08D074
:105CA800334B1B68C3F3C1033248D840E2E732489C
:105CB800C0E73048BEE7402B17D14FF40040626A76
:105CC8002A4B33F81230B0FBF3F0636800EB530053
:105CD800B0FBF3F0A0F110024FF6EF739A4242D8EE
:105CE800236880B2D860002033E0012031E0FDF75E
:105CF8003BFF0028E3D100202BE0FDF747FFF8E742
:105D080003A8FEF7B9FD0498F3E76846FEF7CEFE50
:105D18000198EEE7164B1B6813F0200F08D0144BC0
:105D28001B68C3F3C1031348D840E2E71248C6E72B
:105D38001048C4E701200CE001200AE0012008E037
:105D4800012006E0012004E0012002E0012000E03B
:105D580001200123A4F86A30A4F86830002363679F
:105D6800A36706B070BD0120F3E700BFCC7400083C
:105D7800004402580090D00300093D00836A13F0E4
:105D8800080F06D00268536823F40043816B0B4365
:105D98005360836A13F0010F06D00268536823F436
:105DA8000033C16A0B435360836A13F0020F06D0B5
:105DB8000268536823F48033016B0B435360836A92
:105DC80013F0040F06D00268536823F48023416B54
:105DD8000B435360836A13F0100F06D00268936870
:105DE80023F48053C16B0B439360836A13F0200F35
:105DF80006D00268936823F40053016C0B43936048
:105E0800836A13F0400F0AD00268536823F48013A2
:105E1800416C0B435360436CB3F5801F0BD0836A0E
:105E280013F0800F06D00268536823F40023C16C76
:105E38000B43536070470268536823F4C003816CB6
:105E48000B435360EBE72DE9F84305460E4617462A
:105E58009946DDF820802C68E46936EA04030CBF13
:105E68004FF0010C4FF0000CBC453AD1B8F1FF3FA0
:105E7800F1D0FBF7E1FAA0EB0900404534D8B8F1BE
:105E8800000F33D02B681A6812F0040FE3D0B6F174
:105E9800400218BF0122802EDDD0002ADBD0DA694B
:105EA80012F0080F11D1DA6912F4006FD3D04FF451
:105EB80000621A622846FFF79DF92023C5F8903042
:105EC800002385F8843003200CE008241C6228464F
:105ED800FFF790F9C5F89040002385F88430012039
:105EE80000E00020BDE8F8830320FBE70320F9E782
:105EF8002DE9F04182B01E46D0F88830202B5BD1C6
:105F080004460D469046002A18BF002901D10120F9
:105F180053E00023C0F890302123C0F88830FBF705
:105F28008BFA0746A4F85480A4F85680A368B3F502
:105F3800805F02D04FF0000816E0236943B34FF0AA
:105F4800000811E02023C4F88830032035E038F831
:105F5800023B2268C3F308039362B4F8562092B256
:105F6800013A92B2A4F85620B4F856309BB293B1D5
:105F780000963B46002280212046FFF764FF002858
:105F8800E0D1002DE3D015F8012B23689A62E4E7ED
:105F9800A8460025E8E700963B4600224021204617
:105FA800FFF751FF18B92023C4F8883005E02023F3
:105FB800C4F88830032000E0022002B0BDE8F08178
:105FC8002DE9F04383B01E46D0F88C30202B7ED1CB
:105FD80004460D469046002A18BF002901D1012029
:105FE80076E00023C0F890302222C0F88C20C366E7
:105FF800FBF722FA0746A4F85C80A4F85E80A36841
:10600800B3F5805F06D0A3B9226972B9FF22A4F85C
:10601800602014E0226922B940F2FF12A4F860203F
:106028000DE0FF22A4F8602009E07F22A4F8602098
:1060380005E0B3F1805F0AD00022A4F86020B4F82C
:106048006080B3F5805F0CD04FF0000924E022692E
:106058001AB97F22A4F86020F1E73F22A4F8602053
:10606800EDE7236913B14FF0000915E0A9460025B3
:1060780012E02023C4F88C30032029E023685A6AF0
:106088005FFA88F3134005F8013BB4F85E2092B23A
:10609800013A92B2A4F85E20B4F85E309BB28BB19C
:1060A80000963B46002220212046FFF7CCFE002820
:1060B800DFD1002DE2D123685B6A08EA030329F8DF
:1060C800023BE2E72023C4F88C30002000E00220E5
:1060D80003B0BDE8F08330B583B004460023C0F8B0
:1060E8009030FBF7A9F905462268126812F0080FEC
:1060F80010D123681B6813F0040F28D12023C4F89B
:106108008830C4F88C300020E066206784F884006A
:1061180003B030BD6FF07E430093034600224FF476
:1061280000112046FFF78FFE0028E2D0226852E8CF
:10613800003F23F0800342E800310029F6D12023F4
:10614800C4F88830002384F884300320E0E76FF037
:106158007E4300932B4600224FF480012046FFF730
:1061680072FE0028CAD0226852E8003F23F49073D8
:1061780042E800310029F6D1226802F1080353E809
:10618800003F23F00103083242E800310029F3D12F
:106198002023C4F88C30002384F884300320B7E728
:1061A80078B310B50446D0F888300BB32423C4F86C
:1061B80088302268136823F001031360A36AE3B9E7
:1061C8002046FFF7E1FA012811D02268536823F42A
:1061D800904353602268936823F02A0393602268EF
:1061E800136843F0010313602046FFF774FF10BDE6
:1061F80080F88430FBF70CF8D8E72046FFF7BEFD9F
:10620800DEE7012070470000436E2BB90123A0F898
:106218006A30A0F86830704730B403689A68C2F3EF
:1062280042629968490F094D6B5C1B01084C615C1F
:1062380093FBF1F3A0F86A30AB5C1B01A25C93FB03
:10624800F2F3A0F8683030BC704700BFEC74000867
:10625800E474000870477047704790F88430012B49
:1062680018D0012380F884302423C0F888300368CC
:106278001A68196821F00101196022F00052002300
:10628800436601680A602022C0F8882080F88430BC
:10629800184670470220704738B590F88430012BB3
:1062A8001DD00446012380F884302423C0F88830A8
:1062B80003681D681A6822F001021A600268936870
:1062C80023F0604319439160FFF79EFF23681D6028
:1062D8002023C4F88830002084F8840038BD0220C8
:1062E800FCE738B590F88430012B1DD00446012313
:1062F80080F884302423C0F8883003681D681A6841
:1063080022F001021A600268936823F0606319435F
:106318009160FFF779FF23681D602023C4F8883057
:10632800002084F8840038BD0220FCE7014B18687F
:10633800704700BF1000002470B50D4E0D4D761B40
:10634800B61006D0002455F8043B01349847A642FD
:10635800F9D1094E094D761B01F09CF8B61006D00C
:10636800002455F8043B01349847A642F9D170BD82
:106378000075000800750008087500080075000819
:10638800830730B548D0541E002A3FD0CAB203460E
:1063980001E0013C3AD303F8012B9D07F9D1032C06
:1063A8002DD9CDB245EA05250F2C45EA054536D944
:1063B800A4F1100222F00F0C03F1200EE6444FEA7C
:1063C800121C03F1100242E9045542E90255103249
:1063D8007245F8D10CF1010214F00C0F03EB021214
:1063E80004F00F0C13D0ACF1040323F003030433BF
:1063F800134442F8045B9342FBD10CF003042CB124
:10640800CAB21C4403F8012B9C42FBD130BD644640
:106418001346002CF4D1F9E703461446BFE71A46A1
:10642800A446E0E72DE9F043694CD4F8008083B036
:1064380004460E4617461D46B8F1000F03D0D8F89B
:106448003830002B77D0022F05D0012F00F2AC8016
:10645800002DC0F2A980636EDA0752D52146404666
:1064680000F058F9216B41B104F14003994202D080
:10647800404600F07BFA00232363B4F90CC00023E4
:106488001CF0800FA361636064D12CF44A6C2CF07B
:10649800030C022FA4F80CC06AD001AB6A4621464F
:1064A800404600F095FBA3891843A081002D2FD00A
:1064B800002E2ED0D8F83830002B38D0009B26601C
:1064C800AB42B4F90C301CBF43F40063A381012F25
:1064D80004BF43F00103A3819AB213F00803C4E98F
:1064E80004652CD0D1075DD56D42A561656E00238A
:1064F80015F00105A36027D00025284603B0BDE8A4
:10650800F083A3899B05A9D4A06D00F05DFBA5E7E6
:10651800009D284600F08CFB0646002847D0A3893A
:1065280043F08003A381D8F83830002BC6D1404609
:1065380000F024F9C2E7404600F020F983E7A360A1
:10654800656E15F00105D7D1930524D5284603B00B
:10655800BDE8F0832169404600F008FAB4F90CC0A0
:106568002CF44A6C2CF0030C022FA4F80CC094D124
:106578000025002204F14303A2600122C4E9043289
:106588002360636E4CF0020CD807A4F80CC0DDD46D
:106598001CF4007FDAD1A06D00F018FB284603B088
:1065A800BDE8F083A560CBE74FF0FF35CEE7DDF817
:1065B8000090A94504D0484600F03AFB064620B9A9
:1065C800B4F90CC04FF0FF35D3E74D46A7E700BF3D
:1065D80010000024024B13B1024800F005B87047C0
:1065E80000000000A9680008002301461A46184662
:1065F80000F050BEB1F90C20F8B50C46110707465B
:1066080042D4636842F40062002BA28159DDA56A76
:10661800002D54D000233E683B6093B212F48052A0
:1066280053D1E16901233846A847421C63D0A389A6
:10663800A56A5B0705D56368C01A236B0BB1E36BCA
:10664800C01AE169024600233846A847411C3ED1DA
:106658003B68002B3BD01D2B01D0162B52D1A389B0
:106668002269226023F4006300216160A381216B09
:106678003E6021B304F14003994202D0384600F04D
:1066880075F900202063F8BD2669C6B193B2256864
:1066980026609A070CBF63690023AD1BA3600CE05A
:1066A800D4F824C0E1692B4632463846E047B0F1B9
:1066B800000CA5EB0C05664416DD002DF0DC00206F
:1066C800F8BDE36B002BA2DCF9E7206DB1E7B4F964
:1066D8000C302269226023F40063A3810022DB04CA
:1066E8006260C4D52065C2E7A38943F040034FF038
:1066F800FF30A381F8BD3B68002B98D01D2B06D036
:10670800162B04D0A38943F04003A381F8BD3E6053
:10671800D5E700BF38B50C46054608B1836BA3B171
:10672800B4F90C00B8B1636EDB0701D4810515D547
:1067380028462146FFF75EFF636EDA07054602D456
:10674800A3899B050ED5284638BD00F017F8B4F983
:106758000C000028E7D10546284638BDA06D00F09A
:1067680033FAE5E7A06D00F031FA284638BD00BFDE
:10677800014900F001BA00BF4D7300082DE9F04748
:106788008246394800F020FADAF83840002C66D101
:10679800DAF80450354ACAF83C200323CAE9B8435A
:1067A800DFF8CC90DFF8CC80334F344E04230AF561
:1067B8003B72CAF8E8222146C5E90243C5E900440C
:1067C800C5E904446C660822AC6105F15C00FFF77A
:1067D800D7FDC5E90759C5E90987EE6205F15800F3
:1067E80000F0EEF9DAF80850254BEB602146C5E9D0
:1067F8000044C5E904446C66AC60AC61082205F14C
:106808005C00FFF7BDFDC5E90759C5E90987EE62D8
:1068180005F1580000F0D4F9DAF80C50194BEB6088
:106828002146C5E90044C5E904446C66AC60AC6126
:10683800082205F15C00FFF7A3FD05F15800C5E942
:106848000759C5E90A76C5F8248000F0B9F901238B
:10685800CAF838300448BDE8F04700F0B7B9BDE8D9
:10686800F047014800F0B2B9000A0024796700082F
:10687800E571000809720008497200086972000889
:106888000900010012000200014800F09DB900BF94
:10689800FC090024014800F099B900BFFC09002454
:1068A80038B5084B084D5B1B9C1007D0043B1D44B2
:1068B800013C55F804399847002CF9D1BDE8384017
:1068C80000F0EEBD0C75000808750008F8B5244FF7
:1068D8000C46064600F064FCBA685568C4F57E6349
:1068E8000F3325F003052B4423F47F6323F00F03B4
:1068F800A3F58054B4F5805F07DB0021304600F033
:106908005BFCBB682B44984204D0304600F04EFC38
:106918000020F8BD6142304600F04EFC01300DD039
:10692800104ABB682D1B45F001055D6013683046B1
:106938001B1B136000F03AFC0120F8BD0021304613
:1069480000F03AFCBA68831A0F2BDEDD43F001032E
:106958005360054B03491B68C01A0860D5E700BFA0
:1069680044040024040A00244C080024002961D0AF
:10697800F8B50C46064600F013FC54F8042C7B4F7F
:10698800A4F1080522F0010105EB010CB868DCF858
:106998000430604523F0030300F08B80D207CCF865
:1069A800043032D454F8082CAD1A1144AA6807F1FF
:1069B800080082426AD00CEB0304D4F804E0EC68C7
:1069C800D4601EF0010FA26000F0978041F001032F
:1069D8006B60CCF80010B1F5007F35D27A68CB082F
:1069E80048090121013381401143796007EBC30253
:1069F80057F83310083AC5E9021247F83350CD600A
:106A08003046BDE8F84000F0D1BB0CEB03025268F9
:106A1800D00710D4194407F10800DCF80830834285
:106A280073D0DCF80C20DA60936041F001036B60EE
:106A38006950D0E7704741F00103B1F5007F44F891
:106A4800043CCCF80010C9D3B1F5206F4FEA5123AC
:106A580048D28B0903F1390003F13802C300F81852
:106A6800FB580838984259D05A6822F003028A42E3
:106A780002D99B689842F7D1D868C5E90230856089
:106A8800DD603046BDE8F84000F090BB0CEB030237
:106A98005268D20763D40B44DCE90212CA609160E1
:106AA80043F001026A603046EB50BDE8F84000F060
:106AB8007DBB0B44D10707D454F8082CAD1A1344F6
:106AC800D5E90212CA60916043F001026A60284A5F
:106AD800BD6012689A4293D8264B30461968FFF772
:106AE800F5FE8DE7142B0AD9542B1FD80B0B03F195
:106AF8006F0003F16E02C300B1E719448DE703F19B
:106B08005C0003F15B02C300A9E741F00103C7E998
:106B18000455C5E902006B60695071E77968921005
:106B2800012404FA02F20A437A60A6E7B3F5AA7FC1
:106B380006D8CB0B03F1780003F17702C3008EE788
:106B480040F25452934206D88B0C03F17D0003F1B6
:106B58007C02C30083E74FF47E737E227FE741F017
:106B680001036B60CCF800104AE700BF440400241E
:106B780050080024340A00242DE9F84307468846C3
:106B880000F538764FF00009D6E90154013D11D4DB
:106B9800A389012B05F1FF3508D9B4F90E3001336B
:106BA800214603D03846C04749EA00096B1C04F166
:106BB8006804EDD13668002EE6D14846BDE8F88372
:106BC800704700BF704700BF704700BF704700BFE5
:106BD80070B50C46B1F90E10002996B015461E4640
:106BE80014DB6A4600F014FC00280FDB019A02F45B
:106BF8007042A2F50052B2FA82F24FF48063520951
:106C08004FF4006032602B6016B070BDB4F90C1000
:106C1800002311F08000336004D0402218462A6017
:106C280016B070BD4FF480632B6016B070BD00BF06
:106C3800024B0146186800F003B800BF100000249A
:106C48002DE9F04F01F10B06162E83B0044624D827
:106C5800102900F2BA8000F0A3FA102618220220A8
:106C6800B54F3A44A2F1080153688B4200F0BA804C
:106C78005A68D96822F003021A449D68E9608D6059
:106C8800516841F001012046516003F1080500F008
:106C98008DFA284603B0BDE8F08F36F0070600F1FC
:106CA8009480B14200F2918000F07AFAB6F5FC7F48
:106CB800C0F09A81730A00F08F80042B00F26F8174
:106CC800B30903F1390003F1380CC3009A4F3B4470
:106CD800A3F108055B689D4206D10CE0002980F20B
:106CE8002781DB689D4206D05A6822F00302911B77
:106CF8000F29F3DD60463D69DFF840C265457CD069
:106D08006A6822F00302931B0F2B00F37B81002B90
:106D1800C7E904CC80F26C81B2F5007F80F01A815B
:106D2800D308796801334FEA521E012202FA0EF2A3
:106D38000A4357F833E0C5F808E007EBC301083900
:106D4800E9607A6047F83350CEF80C50831001217F
:106D58009940914257D8114206D120F003004900CA
:106D6800114200F10400FAD007EBC0094D468646EF
:106D7800D5F80C80454508D11DE1002B80F224810F
:106D8800D8F80C80454500F01681D8F8042022F088
:106D98000302931B0F2BF0DD2046D8E9025408EBC1
:106DA800060146F00106C8F80460EC60A56043F0EF
:106DB8000104C7E90411C1E902CC4C6048F802306B
:106DC80000F0F4F908F1080502E00C23236000251F
:106DD800284603B0BDE8F08F4FF4007340204FF011
:106DE8003F0C73E7D3689A4208BF02307FF440AF84
:106DF8003D69DFF848C1654582D17A688310012171
:106E080099409142A7D9BD686B6823F003094E45A4
:106E180003D8A9EB06030F2B7ADCDFF824B1494B22
:106E2800DBF800201B680132334405EB090A00F047
:106E3800338103F580530F3323F47F6828F00F085C
:106E48004146204600F0B8F9411C024600F0F380A4
:106E5800824500F2EE803C4B1968414419600846AF
:106E680000F04E81DBF80010019301311BBFA2EB4B
:106E78000A0A5044CBF80020186012F0070B00F003
:106E88001781CBF108010A44CBF5805190440831B1
:106E9800A1EB0801C1F30B0A51462046009200F00D
:106EA8008BF9421CDDE9002300F04F81801A00EBCA
:106EB8000A081968BA6048F001005144BD425060A0
:106EC800196000F02981B9F10F0F40F22781686835
:106ED800A9F10C0C2CF0070C00F0010040EA0C00A2
:106EE80068604FF0050E05EB0C00BCF10F0FC0E910
:106EF80001EE00F2328150681546144B1A688A4236
:106F080038BF1960124B1A688A4238BF196094E07A
:106F1800AA1943F0010346F001066E602046BA60E4
:106F2800536000F043F90835284603B0BDE8F08FF8
:106F3800D9681A44A1E600BF440400244C04002484
:106F48004C080024340A0024040A00242C0A0024D3
:106F5800300A0024B2F5206F4FEA522363D3142B72
:106F680000F2B78003F15C01C9005B3307EB010E47
:106F78007958AEF1080E8E4500F091804B6823F0E9
:106F88000303934202D989688E45F7D1D1F80CE002
:106F98007A68C5E9021ECEF80850CD60D6E6142BF3
:106FA80059D9542B00F29D80330B03F16F0003F184
:106FB8006E0CC3008AE60EF1010E1EF0030F05F1F8
:106FC80008057FF4D5AE51E0424445465368D8F8E9
:106FD8000C1043F00103536055F8083F2046D96070
:106FE8008B6000F0E3F8F3E6F00806F1080237E6F4
:106FF8002A442046536843F001035360083500F0E3
:10700800D5F8E5E6A919204646F0010643F0010443
:107018006E60C7E90411C1E902CC4C60AB5000F0C6
:10702800C5F80835D4E6930903F13901C9003833A6
:107038009CE7BD425FD0BD68686820F003084645FC
:10704800A8EB060302D80F2B3FF762AF204600F0EB
:10705800ADF80025BCE603F15C0003F15B0CC3004E
:1070680034E659F808394B4540F0968010F0030F84
:1070780000F1FF30F5D17B6823EA01037B6049000A
:1070880099423FF6C0AE19B9BDE649000EF1040EAB
:107098001942FAD0704667E603F11008D0E69A1054
:1070A8004FF001087B6808FA02F21A437A6070E729
:1070B80002EB08014942C1F30B0A514620460092EF
:1070C80000F07AF8431CDDE900237FF4EFAEDA46DE
:1070D800EFE6542B25D8130B03F16F01C9006E336B
:1070E80044E7B3F5AA7F25D8F30B03F1780003F141
:1070F800770CC300EAE5294B186840441860B1E6EC
:10710800CAF30B0CBCF1000F7FF4ACAEBD68C844E9
:1071180048F001006860F0E61546EEE6012353608A
:1071280094E7B3F5AA7F23D8D30B03F17801C900FC
:1071380077331BE740F25452934223D8B30C03F140
:107148007D0003F17C0CC300C0E5ABF1080BD8440B
:10715800A8EB02084FF0000AABE605F1080120464B
:107168000093FFF703FCBD68009B68681968C4E6D4
:1071780040F254518B420BD8930C03F17D01C900A6
:107188007C33F3E64FF47E737F204FF07E0C9DE551
:107198004FF47E717E23E9E67B6870E7040A0024D9
:1071A8000148FFF711BD00BFF80900240148FFF7A7
:1071B8000DBD00BFF809002438B5074D002204466C
:1071C80008462A60F9F7FCFE431C00D038BD2B683E
:1071D800002BFBD0236038BD380A002410B50C46BC
:1071E800B1F90E1000F040F9002803DB236D0344C9
:1071F800236510BDA38923F48053A38110BD00BF6C
:107208002DE9F0410C46B1F90C101F46CB05054697
:1072180016460BD421F48051A1813B46B4F90E10D7
:1072280032462846BDE8F04100F01EB8B4F90E1009
:107238000223002200F002F9B4F90C10EAE700BFBB
:1072480010B50C46B1F90E1000F0F8F8A389421CED
:107258000EBF23F4805343F480532065A38110BDEF
:10726800B1F90E1000F05CB838B50C46084D8446EC
:10727800114620461A4600232B606446F9F704FE9F
:10728800431C00D038BD2B68002BFBD0236038BDD1
:10729800380A00242DE9F047DFF87CA00646DAF822
:1072A800000098460F469146FFF78EFC1B4B1B6863
:1072B800D3F8484124B365681F2D26DC5EB96B1CE2
:1072C8000235DAF80000636044F82570FFF77EFCA9
:1072D8000020BDE8F08704EB85010123C1F8889000
:1072E800D4F88821AB401A43022EC4F88821C1F88B
:1072F8000881E4D1D4F88C211343C4F88C31DEE73B
:1073080003F5A674C3F84841D5E7DAF80000FFF79B
:107318005DFC4FF0FF30DCE740040024F474000803
:1073280038B5074D0022044608462A60F9F7C6FD1D
:10733800431C00D038BD2B68002BFBD0236038BD20
:10734800380A002470B500294BD006460C4610B107
:10735800836B002B48D0636ED80734D5B4F90C3052
:10736800002B3ED021463046FFF744F9E36A054634
:1073780033B1E169304698470028B8BF4FF0FF3570
:10738800A3891A063BD4216B41B104F14003994209
:1073980002D03046FFF7EAFA00232363616C21B17B
:1073A8003046FFF7E3FA00236364FFF76DFA636E74
:1073B8000022DB07A28127D5A06DFFF703FCFFF7AA
:1073C80069FA284670BDA3899905CBD4A06DFFF74B
:1073D800FBFBB4F90C30002BC4D1656E15F0010528
:1073E80008D00025284670BDFFF7C8F9636ED80796
:1073F800B4D4E8E7A06DFFF7E9FB284670BD216922
:107408003046FFF7B3FABEE7A06DFFF7DFFBD3E71F
:1074180070B50C46084D03460026204611461C460A
:107428002E60F9F777FD431C00D070BD2B68002B48
:10743800FBD0236070BD00BF380A002438B50C4665
:10744800084D8446114620461A4600232B606446A0
:10745800F9F740FD431C00D038BD2B68002BFBD04A
:10746800236038BD380A002438B50C46084D8446D8
:10747800114620461A4600232B606446F9F732FD70
:10748800431C00D038BD2B68002BFBD0236038BDCF
:10749800380A0024F8B500BFF8BC08BC9E467047FF
:0C74A800F8B500BFF8BC08BC9E46704759
:1074B4000000000001020304010203040607080996
:1074C4000006101600061016010002000400060053
:1074D40008000A000C001000200040008000000199
:1074E400080402040801010101010103070100006D
:0474F4001800002458
:0874F8000C93FF7F010000006E
:08750000DD650008BD02000872
:0475080099020008DC
:10750C000090D0030090D003010000001000000098
:10751C0018000024000000000000000004030024F8
:10752C006C030024D40300240000000000000000C1
:10753C00000000000000000000000000000000003F
:10754C00000000000000000000000000000000002F
:10755C00000000000000000000000000000000001F
:10756C00000000000000000000000000000000000F
:10757C0000000000000000000000000000000000FF
:10758C0000000000000000000000000000000000EF
:10759C0000000000000000000000000000000000DF
:1075AC0000000000000000000000000000000000CF
:1075BC0000000000000000000000000000000000BF
:1075CC0001000000000000000E33CDAB34126DE65C
:1075DC00ECDE05000B0000000000000000000000C5
:1075EC00000000000000000000000000000000008F
:1075FC00000000000000000000000000000000007F
:10760C00000000000000000000000000000000006E
:10761C00000000000000000000000000000000005E
:10794C00F40900240000000000000000440400249E
:10795C00440400244C0400244C040024540400244B
:10796C00540400245C0400245C04002464040024FB
:10797C00640400246C0400246C04002474040024AB
:10798C00740400247C0400247C040024840400245B
:10799C00840400248C0400248C040024940400240B
:1079AC00940400249C0400249C040024A4040024BB
:1079BC00A4040024AC040024AC040024B40400246B
:1079CC00B4040024BC040024BC040024C40400241B
:1079DC00C4040024CC040024CC040024D4040024CB
:1079EC00D4040024DC040024DC040024E40400247B
:1079FC00E4040024EC040024EC040024F40400242B
:107A0C00F4040024FC040024FC04002404050024D9
:107A1C00040500240C0500240C0500241405002486
:107A2C00140500241C0500241C0500242405002436
:107A3C00240500242C0500242C05002434050024E6
:107A4C00340500243C0500243C0500244405002496
:107A5C00440500244C0500244C0500245405002446
:107A6C00540500245C0500245C05002464050024F6
:107A7C00640500246C0500246C05002474050024A6
:107A8C00740500247C0500247C0500248405002456
:107A9C00840500248C0500248C0500249405002406
:107AAC00940500249C0500249C050024A4050024B6
:107ABC00A4050024AC050024AC050024B405002466
:107ACC00B4050024BC050024BC050024C405002416
:107ADC00C4050024CC050024CC050024D4050024C6
:107AEC00D4050024DC050024DC050024E405002476
:107AFC00E4050024EC050024EC050024F405002426
:107B0C00F4050024FC050024FC05002404060024D4
:107B1C00040600240C0600240C0600241406002481
:107B2C00140600241C0600241C0600242406002431
:107B3C00240600242C0600242C06002434060024E1
:107B4C00340600243C0600243C0600244406002491
:107B5C00440600244C0600244C0600245406002441
:107B6C00540600245C0600245C06002464060024F1
:107B7C00640600246C0600246C06002474060024A1
:107B8C00740600247C0600247C0600248406002451
:107B9C00840600248C0600248C0600249406002401
:107BAC00940600249C0600249C060024A4060024B1
:107BBC00A4060024AC060024AC060024B406002461
:107BCC00B4060024BC060024BC060024C406002411
:107BDC00C4060024CC060024CC060024D4060024C1
:107BEC00D4060024DC060024DC060024E406002471
:107BFC00E4060024EC060024EC060024F406002421
:107C0C00F4060024FC060024FC06002404070024CF
:107C1C00040700240C0700240C070024140700247C
:107C2C00140700241C0700241C070024240700242C
:107C3C00240700242C0700242C07002434070024DC
:107C4C00340700243C0700243C070024440700248C
:107C5C00440700244C0700244C070024540700243C
:107C6C00540700245C0700245C07002464070024EC
:107C7C00640700246C0700246C070024740700249C
:107C8C00740700247C0700247C070024840700244C
:107C9C00840700248C0700248C07002494070024FC
:107CAC00940700249C0700249C070024A4070024AC
:107CBC00A4070024AC070024AC070024B40700245C
:107CCC00B4070024BC070024BC070024C40700240C
:107CDC00C4070024CC070024CC070024D4070024BC
:107CEC00D4070024DC070024DC070024E40700246C
:107CFC00E4070024EC070024EC070024F40700241C
:107D0C00F4070024FC070024FC07002404080024CA
:107D1C00040800240C0800240C0800241408002477
:107D2C00140800241C0800241C0800242408002427
:107D3C00240800242C0800242C08002434080024D7
:107D4C00340800243C0800243C080024FFFFFFFFFB
:047D5C000000020021
:0400000508001329B3
:00000001FF
